:100000000C9407040C942F040C942F040C942F04CC
:100010000C942F040C942F040C9467370C942F0429
:100020000C942F040C942F040C942F040C942F0484
:100030000C942F040C942F040C94BB380C946C3942
:100040000C942F040C942F040C942F040C942F0464
:100050000C94F8360C942F040C942F040C942F0459
:100060000C941D370C9424380C94B2370C948C37B4
:100070000C942F040C94AE360C942F040C942F0483
:100080000C942F040C942F040C9442370C94D33608
:100090000C944A360C94FE370C94D8370C942F04E9
:1000A00007634236B79BD8A71A39685618AEBAAB61
:1000B000558C1D3CB7CC5763BD6DEDFD753EF617F5
:1000C0007231BF000000803F08000000BE9224494A
:1000D000123EABAAAA2ABECDCCCC4C3E000000807A
:1000E000BEABAAAAAA3E00000000BF000000803FED
:1000F0000000000000084178D3BB4387D1133D19AD
:100100000E3CC3BD4282AD2B3E68EC8276BED98FD9
:10011000E1A93E4C80EFFFBE01C4FF7F3F0000001D
:100120000000010008191304E81A0010191302E86E
:100130004C0011191301E8820010191301E8B400F2
:1001400011191301E8EA0010191302E81C01101933
:100150001302E84E0111191301E8000303070F3FD2
:10016000FFFF07070707070707070707070707072F
:100170000707070707E01FF83FFC7C3E700FF00FF2
:10018000E007E00700070007000F001E003C00F832
:1001900003F007C01F003C00380070006000E00062
:1001A000FFFFFFFFFFFF07F007FE07FF8783C38006
:1001B000F38039C01CE00E0007000F007F003F00F5
:1001C0001FE00078001E00070003F001F800FE00A9
:1001D000770073E0F8FFF83FF807F00000380038C8
:1001E000007800F800F801F803B8033807380E3833
:1001F0001C381838383870386038E038FFFFFFFF97
:10020000FFFF0038003800380038003800381FFF82
:100210000FFF8FFFC700038001C000E000700039AE
:10022000F03FFE1FFF8F83E700F0003C000E000749
:1002300000038001C000FC00EF0073C0F0FFF83F36
:10024000F807E00003E00FF81FFC3C1E380E700EAC
:1002500070006000E000E3E0EFF8FFFCFC3EF00E11
:10026000F00FE007E007E0076007700F700E3C3EFC
:100270003FFC1FF807E0FFFFFFFFFFFF0006000E37
:10028000001C001800380070006000E000C001C0D1
:100290000180038003800700070007000E000E00A6
:1002A0000E000C001C001C0007F00FFE0FFF8783E0
:1002B000C780F38039C01CE00E780F1E0F07FF01C6
:1002C000FF03FFE3E0F9C01DC00FE003F001F800F9
:1002D000FC00F70073E0F8FFF83FF807F000005A61
:1002E000012201310038003800000000003E5B4F61
:1002F0005B3E3E6B4F6B3E1C3E7C3E1C183C7E3C86
:10030000181C577D571C1C5E7F5E1C00183C180093
:10031000FFE7C3E7FF0018241800FFE7DBE7FF3023
:10032000483A060E2629792926407F050507407F91
:1003300005253F5A3CE73C5A7F3E1C1C08081C1C04
:100340003E7F14227F22145F5F005F5F06097F01FA
:100350007F006689956A606060606094A2FFA294E5
:1003600008047E040810207E201008082A1C0808B3
:100370001C2A08081E101010100C1E0C1E0C303801
:100380003E3830060E3E0E06000000000000005F02
:1003900000000007000700147F147F14242A7F2A1E
:1003A00012231308646236495620500008070300E0
:1003B000001C2241000041221C002A1C7F1C2A082C
:1003C000083E08080080703000080808080800008F
:1003D00060600020100804023E5149453E00427F03
:1003E000400072494949462141494D331814127F52
:1003F0001027454545393C4A4949314121110907F2
:100400003649494936464949291E00001400000072
:100410004034000000081422411414141414004144
:1004200022140802015909063E415D594E7C121101
:10043000127C7F494949363E414141227F41414139
:100440003E7F494949417F090909013E41415173B4
:100450007F0808087F00417F41002040413F017F25
:10046000081422417F404040407F021C027F7F04ED
:1004700008107F3E4141413E7F090909063E415136
:10048000215E7F09192946264949493203017F0126
:10049000033F4040403F1F2040201F3F4038403F27
:1004A000631408146303047804036159494D43003D
:1004B0007F4141410204081020004141417F040274
:1004C000010204404040404000030708002054540B
:1004D00078407F28444438384444442838444428E9
:1004E0007F385454541800087E090218A4A49C783C
:1004F0007F0804047800447D40002040403D007F98
:100500001028440000417F40007C047804787C0877
:100510000404783844444438FC182424181824244B
:1005200018FC7C08040408485454542404043F4430
:10053000243C4040207C1C2040201C3C4030403C5F
:1005400044281028444C9090907C4464544C4400BF
:100550000836410000007700000041360800020123
:100560000204023C2623263C1EA1A161123A40400F
:10057000207A38545455592155557941225454788C
:1005800042215554784020545579400C1E52721225
:1005900039555555593954545459395554545800AE
:1005A00000457C410002457D420001457C407D12B2
:1005B00011127DF0282528F07C5455450020545414
:1005C0007C547C0A097F4932494949323A444444BF
:1005D0003A324A4848303A4141217A3A42402078FA
:1005E000009DA0A07D3D4242423D3D4040403D3CFB
:1005F00024FF2424487E4943662B2FFC2F2BFF0920
:1006000029F620C0887E0903205454794100004413
:100610007D413048484A32384040227A007A0A0AFE
:10062000727D0D19317D2629292F28262929292671
:1006300030484D4020380808080808080808382FB6
:1006400010C8ACBA2F102834FA00007B0000081440
:100650002A142222142A14085500550055AA55AA16
:1006600055AAFF55FF55FF000000FF00101010FFB6
:1006700000141414FF001010FF00FF1010F010F011
:10068000141414FC001414F700FF0000FF00FF1402
:1006900014F404FC141417101F10101F101F14144E
:1006A000141F00101010F0000000001F1010101098
:1006B0001F10101010F010000000FF10101010108C
:1006C00010101010FF10000000FF140000FF00FFCA
:1006D00000001F10170000FC04F414141710171466
:1006E00014F404F40000FF00F71414141414141488
:1006F000F700F7141414171410101F101F141414FB
:10070000F4141010F010F000001F101F0000001F64
:1007100014000000FC140000F010F01010FF10FF97
:10072000141414FF141010101F00000000F010FF2C
:10073000FFFFFFFFF0F0F0F0F0FFFFFF0000000010
:1007400000FFFF0F0F0F0F0F3844443844FC4A4A94
:100750004A347E02020606027E027E026355494149
:10076000633844443C04407E201E2006027E020280
:1007700099A5E7A5991C2A492A1C4C7201724C3094
:100780004A4D4D303048784830BC625A463D3E496B
:100790004949007E0101017E2A2A2A2A2A44445F0F
:1007A000444440514A444040444A51400000FF0103
:1007B00003E080FF000008086B6B08361236243611
:1007C000060F090F06000018180000001010003076
:1007D00040FF0101001F01011E00191D1712003CFE
:1007E0003C3C3C00000000000901809611800A3A60
:1007F00081550A3601082A04000000F02B0400008D
:10080000014021800A13800A29800A002C3A112411
:100810001FBECFEFCDBFDFE3DEBF18E2A0E0B8E23E
:10082000E5EAF1EB02C005900D92A637B107D9F7C2
:100830002EE2A6E7B8E201C01D92A431B207E1F7AB
:1008400014E0C7E0D4E004C02197FE010E94BA552D
:10085000C630D107C9F70E94B93B0C9422570C94BB
:10086000000090E0FC01E85BF041E081EF3F39F1EE
:1008700084529041DC012C91822F880F880F880FC1
:100880008E0F8033E0F490E0880F991FDC01A75BA6
:10089000B44D6D937C938751954DDC011D921C9254
:1008A000B0E22B9FC00111249C5F4096E80FF92F06
:1008B000F11D8081887F808380818160808308959D
:1008C000CF93DF93EC0189819A81DC01ED91FC915A
:1008D0000280F381E02D41E050E00995019761F439
:1008E00089819A81DC01ED91FC91008CF18DE02DE4
:1008F00061E0099591E0811190E0892FDF91CF911E
:100900000895FC0154894589252F30E0842F90E01B
:10091000821B930B541710F0CF96089501970895FA
:10092000FC0192898389981761F0A389AE0FBF2FCC
:10093000B11D59968C9193899F5F9F73938B90E023
:1009400008958FEF9FEF0895FC019289838998178E
:1009500031F08389E80FF11D818D90E008958FEFCC
:100960009FEF0895FC0192892389892F90E0805C94
:100970009F4F821B91098F7399270895CF93DF931F
:10098000EC01E881F9810680F781E02D0995EC857D
:10099000FD8586818F738683EC85FD8585818F75C6
:1009A00085838B898A8B198ADF91CF910895CF93A4
:1009B000DF93FC0194898589C485D585981306C089
:1009C0008D818F7D8D83DF91CF910895A589AE0FA5
:1009D000BF2FB11DA75ABF4F2C91858990E001967A
:1009E0008F739927858B80E48C83A485B5851296B7
:1009F0002C93948985899813E6CFA485B58515969F
:100A00008C9115978F7D15968C9387898823D9F2C1
:100A1000808D80931301178AD6CFDC011C96ED914F
:100A2000FC910FB607FE03C0258125FD04C024817B
:100A300025FD0C94D7040895EF92FF920F931F9316
:100A4000CF93DF93EC0181E0898B9C898D8998138A
:100A50001CC0AC85BD8514968C91149785FF15C07C
:100A600012966C93AC85BD8580E414968C93EC85CE
:100A7000FD8585818F7D858381E090E0DF91CF9139
:100A80001F910F91FF90EF9008958091110180FFC9
:100A900008C080911301888F8E898093130181E0B3
:100AA0008F8BF62E0C8910E00F5F1F4F0F731127ED
:100AB000E02E8D898E1104C0CE010E940D05F9CF64
:100AC000EC89EC0FFD2FF11DE75AFF4FF0820C8BE4
:100AD000EC85FD8585818062CECFCF93DF93FC01CD
:100AE00021892223C9F0EC018091110180FF08C007
:100AF00080911301808F86898093130181E0878B19
:100B0000EC85FD85858185FD03C0848186FD04C05B
:100B1000CE010E940D05F4CFDF91CF910895CF93C0
:100B2000DF9390E0FC01EE53F04120812F3F89F0EC
:100B30006330710570F4FC01E452F041A08130E2B1
:100B4000A39FD0011124BC5F6130710529F4119677
:100B50002C93DF91CF910895885B9041EC01E8815F
:100B6000EF3F89F0CD014096E80FF92FF11D9FB7B7
:100B7000F89412962C9380816230710539F4886064
:100B800080839FBFE6CFF0E0E0E0F1CF877FF8CF32
:100B9000282F30E0F901E65EF041E081EE2309F113
:100BA000E13021F0F0F0E63098F008954091010A2C
:100BB000285B3041F90120812C5F81E090E001C089
:100BC000880F2A95EAF7809584238093010A089577
:100BD00080E1E89FF0011124E05AF54F81818F7E7A
:100BE00081830895FF920F931F93CF93DF93082F74
:100BF00010E0F801EE53F041F0809FEFF916A1F0FC
:100C0000EB018B3210F40E94C805F801E452F04168
:100C1000E08180E2E89FF0011124FC5F80818F2158
:100C200059F0CD2B39F4F682DF91CF911F910F91BE
:100C3000FF900895F582F8CFD801A85BB0418C9160
:100C4000309771F08F3F61F07096E80FF11D9FB7FC
:100C5000F8948081CD2B39F4877F80839FBFE4CFC8
:100C6000F0E0E0E0F4CF8860F8CF0F931F93CF93CC
:100C7000082F10E0F801EE53F041C081CF3FB9F0EA
:100C80008B3210F40E94C805F801E452F041E08173
:100C900080E2E89FF0011124FC5F8085C82381E099
:100CA00090E009F480E0CF911F910F91089580E0CA
:100CB00090E0F9CF8B3210F40C94F20508958B324A
:100CC00010F40C948F050895CF92DF92EF92FF926B
:100CD0000F931F93CF93DF93EC016A017B01022FE7
:100CE0008989882339F0E881F9810288F389E02D28
:100CF000CE01099598898091E205892B8093E205C0
:100D00001FB7F89460E070E281EA97E0A7019601CE
:100D10000E94285169017A018FEFC81AD80AE80A9F
:100D2000F80AF694E794D794C794EC85FD858681FC
:100D30008D7F8683EC85FD8586818683198AA091C7
:100D400023110A2E000CBB0BA70196010E94EF5045
:100D500020E034E040E050E00E94C550EC85FD8585
:100D6000C20ED31EE41EF51EC086D186EC85FD851D
:100D70000783EC85FD858681806C8683EC85FD8507
:100D80008581806885838E8562E070E00E945F06C1
:100D90008F8561E070E00E945A068F8561E070E007
:100DA0000E945F061FBFDF91CF911F910F91FF90AF
:100DB000EF90DF90CF900895E82FF0E0EE5EF041E5
:100DC0008E30B8F480818F30B0F48093060681E0D5
:100DD0008093080680910B0680FFFCCF2FB7F89414
:100DE00090911006809111062FBF89279827892797
:100DF00008953E97E7CF8FEF90E00895CF93DF936C
:100E00008FB7F8942091E02A3091E12A4091E22AAC
:100E10005091E32AE091BA0A9091B60A90FF06C079
:100E20002F5F3F4F4F4F5F4FE091BA0A8FBFA091A6
:100E3000DE2AB091DF2AC091DC2AD091DD2A0E94FF
:100E4000E450EC9F9001ED9F300D1124620F731F51
:100E5000811D911DDF91CF9108958F929F92AF9246
:100E6000BF92CF92DF92EF92FF924B015C010E9402
:100E7000FE066B017C01A8EEB3E0A50194010E947F
:100E8000E450C60ED71EE81EF91EC616D706E806A1
:100E9000F90618F40E94FE06F8CF0E94FE066C15B3
:100EA0007D058E059F05C8F3FF90EF90DF90CF90F2
:100EB000BF90AF909F908F9008952FB7F894609156
:100EC000D82A7091D92A8091DA2A9091DB2A2FBFF3
:100ED00008950F931F93CF93DF938C01EB018091C3
:100EE0005C2890915D28A0915E28B0915F28892BA5
:100EF0008A2B8B2B51F40E945D0760935C287093C2
:100F00005D2880935E2890935F280130110539F0A9
:100F1000CF3FDC07A1F481E08093612806C0CF3F7A
:100F2000DC0741F481E080936028DF91CF911F912D
:100F30000F910895C0936528D0936628F6CFC0938B
:100F40006328D0936428F1CF7F928F929F92AF92C3
:100F5000BF92CF92DF92EF92FF920F931F93CF93A6
:100F6000DF93782EEB017A010091C22D1091C32DF1
:100F7000D8011496CD90DC9021E0C114D10409F47D
:100F800020E0822E912CF80181819281DC01ED918B
:100F9000FC91048CF58DE02DA401D8016C9109958C
:100FA00088159905D1F480ECA82E8DE2B82EC501E4
:100FB000805C9D428815990570F4F80181819281C9
:100FC000DC01ED91FC910284F385E02D0995F5019A
:100FD00081935F01ECCFCD2859F20091C02D10E034
:100FE00002C0159507957A94E2F7017011270E94C7
:100FF0005D07012B09F059C088809980AA80BB80C9
:1010000081149104A104B10431F4688379838A8343
:101010009B8310E024C01D811111FBCF6819790951
:101020008A099B096D3271408105910598F081E034
:101030008D838F8198858230910508F459C0843062
:10104000910508F066C02D81222309F46EC081E06D
:101050008E835FC08C81811102C081E08C838F817F
:1010600098850297029790F4112381F0D701179683
:101070008D919C9118970297029740F419968D9143
:101080009C911A9717968D939C931897812FDF91B7
:10109000CF911F910F91FF90EF90DF90CF90BF9075
:1010A000AF909F908F907F9008951C811123C1F085
:1010B0002D81211114C088809980AA80BB80681975
:1010C00079098A099B0989889A88092C000CAA0841
:1010D000BB0886169706A806B90608F4AACF10E042
:1010E0001C821D821E82188219821A821B82B7CF2F
:1010F00089879A872D81222399F0019771F083E0E7
:1011000090E08F8398870E945D076B877C878D872F
:101110009E871111E5CF11E0A2CF82E090E0F1CFE0
:1011200021E082278F839887F4CF29853A858987A4
:101130009A872F833887EDCFAF92BF92CF92DF92FD
:10114000EF92FF920F931F93CF93DF936C017B017C
:101150008B01040F151FEB015E01AE18BF08C0170D
:10116000D10759F06991D601ED91FC910190F08180
:10117000E02DC6010995892B79F7C501DF91CF9143
:101180001F910F91FF90EF90DF90CF90BF90AF90A5
:101190000895EF92FF920F931F93CF93DF93C82F81
:1011A000D0E0A09695E0CC0FDD1F9A95E1F7E98499
:1011B000F82EFF0CFF0CFF0C01E010E08E2D8023B9
:1011C000A9F02F2D210F30E0220F331FF901E75B2B
:1011D000F44D80819181892B49F00190F081E02DBF
:1011E0002751354DD9018D919C9109951F5F000FB5
:1011F000183021F7E986DF91CF911F910F91FF9071
:10120000EF900895FC01A485B58511968C911197F6
:1012100081FD1BC06C9182898F5F8F7393899817B2
:1012200039F0A289AE0FBF2FB11D59966C93828BF6
:10123000E756FF4F80819181009741F0DC01ED91ED
:10124000FC910190F081E02D09948C91089581E04A
:101250000895FC019085957081E0953009F080E05B
:101260000895CF92DF92EF92FF920F931F93CF9347
:10127000DF93EC0188858B7F8887E881F981019075
:10128000F081E02DCE010995182F88858695817013
:101290001817B9F00E945D076A837B838C839D8356
:1012A000888592E089278887888582FB882780F94E
:1012B000DF91CF911F910F91FF90EF90DF90CF9032
:1012C00008950E945D07CA80DB80EC80FD80AB0141
:1012D000BC014C195D096E097F098E819F81B0E0C8
:1012E000A0E0481759076A077B07F0F288858170EC
:1012F0001817D1F20E945D076A837B838C839D83DC
:10130000888591E08927846088870E945D07098528
:101310001A852B853C85601B710B820B930B6D87A7
:101320007E878F87988B0E945D0769877A878B8776
:101330009C87BACFCF93DF93EC011886E881F981BF
:101340000190F081E02D0995882319F0888583604C
:1013500088870E945D076A837B838C839D83DF91EE
:10136000CF910895862FBA010C945F06FC01818904
:1013700030E020E08B3218F40E9435069C0181E0B9
:10138000232B09F480E008950895EF92FF920F93C4
:101390001F93CF93DF937C01EB018B01040F151F8B
:1013A000C017D10759F0D701ED91FC910480F58168
:1013B000E02D6881C70109958993F2CFDF91CF9124
:1013C0001F910F91FF90EF9008950F931F93CF936C
:1013D000DF93EC018B018091C008E881F9810480E2
:1013E000F581E02D86FD13C0612FCE010995182FE0
:1013F000E881F9810480F581E02D602FCE01099507
:10140000082FC801DF91CF911F910F910895CE0150
:101410000995082FE881F9810480F581E02D612F7D
:10142000CE010995182FEDCF00006093C40880917C
:10143000C30887FFFCCF8091C40808958F929F92C4
:10144000AF92BF92CF92DF92EF92FF920F931F93D2
:10145000CF93DF93FC018085882319F081FF0EC0B4
:101460007894DF91CF911F910F91FF90EF90DF90D3
:10147000CF90BF90AF909F908F90089580FFF1CF55
:1014800082849384A484B584C12CD12C760110E08D
:101490009401A501B601C701A0E00E94EC5599F1A5
:1014A000217030E040E050E060E070E080E090E0EB
:1014B0000E94EC55D9F0D0E0C0E0103370F4C12F99
:1014C000C695C695C69580E2C89FE0011124C05F0D
:1014D000DB4F812F8770C80FD11DCF01810F911D68
:1014E000DC0152968C919881892B88839401A50107
:1014F000B601C70101E00E94D15549015A016B01B3
:101500007C011F5FC5CF86849784A088B188C12CD9
:10151000D12C760110E29401A501B601C701A0E02B
:101520000E94EC5509F49DCF217030E040E050E07E
:1015300060E070E080E090E00E94EC55D9F0D0E0EF
:10154000C0E0103370F4C12FC695C695C695B0E2C1
:10155000CB9FE0011124C05FDB4F812F8770C80F44
:10156000D11DCF01810F911DDC0152968C91988184
:10157000892B88839401A501B601C70101E00E946F
:10158000D15549015A016B017C011F5FC4CFFC0199
:101590006F3F710581F1808581FD2DC0603271053D
:1015A0005CF581E090E002C0880F991F6A95E2F730
:1015B00080959095092E000CAA0BBB0B4285538594
:1015C0006485758584239523A623B7238287938713
:1015D000A487B58782859385A485B585892B8A2BB9
:1015E0008B2B49F486859785A089B189892B8A2B15
:1015F0008B2B09F4108608956052710981E090E008
:1016000002C0880F991F6A95E2F780959095092E80
:10161000000CAA0BBB0B4685578560897189842312
:101620009523A623B72386879787A08BB18BD2CF2C
:10163000FC016F3F7105E9F1603371051CF082E038
:101640008087089580858160808760327105C4F449
:1016500081E090E002C0880F991F6A95E2F7092E99
:10166000000CAA0BBB0B4285538564857585842BC2
:10167000952BA62BB72B82879387A487B5870895D0
:101680006052710981E090E002C0880F991F6A954D
:10169000E2F7092E000CAA0BBB0B46855785608923
:1016A0007189842B952BA62BB72B86879787A08BC8
:1016B000B18B0895E0ECF8E020812E7F2083FC01BF
:1016C00017820895E0ECF8E082818E7F828308958E
:1016D000E0ECF8E082818160828308950F9391E0CD
:1016E0009093422A1092412A60933F2A7093402A95
:1016F00040933E2A20933D2A10923C2A10923B2A86
:1017000000933A2A880F8093392A23E030E044E09E
:1017100050E080913E2A882341F02093372A30936D
:10172000382A8091392A8E7F0BC080913D2A8823E8
:1017300051F04093372A5093382A8091392A81609A
:101740008093A70808C080913E2A811104C080912F
:101750003D2A882311F38091412A8823E1F3809167
:10176000412A8330B1F280913D2A882321F0809173
:101770003B2A0F9108958091412A823031F08530C3
:1017800031F0813031F480E0F4CF81E0F2CF83E0BA
:10179000F0CF84E0EECFE0EAF8E0918590669187A3
:1017A00022E030E02093372A3093382A8093292A88
:1017B0001092282A089581E08093282A1092292ADD
:1017C00093E09093AA089091AB0891FF10C01092FB
:1017D000352AE091262AF091272A09958093342A08
:1017E00085E090E08093372A9093382A08951092EC
:1017F000362A8093332A86E090E0F4CF8F929F922E
:10180000AF92BF92CF92DF92EF92FF92CF93DF938E
:1018100060342DE0720723E08207910508F454C07C
:10182000611525E372072CE08207910508F445C095
:1018300060387F448241910508F046C0C8E7D0E097
:1018400020E432E44FE050E080901128909012287C
:10185000A0901328B0901428C501B4010E9428510B
:1018600069017A018AE0C81AD108E108F108C501C6
:10187000B40120E432E44FE050E00E942851DE0140
:101880000E94E45028EE33E040E050E00E942851EE
:10189000C21AD30AE40AF50AF694E794D794C794D7
:1018A000C092A608DF91CF91FF90EF90DF90CF908C
:1018B000BF90AF909F908F900895CCE2D1E020E848
:1018C0003AE146E050E0C0CFC8EED3E020EA36E887
:1018D00041E050E0B9CF6093242A7093252A0895FF
:1018E0006093222A7093232A0895E091242AF0918C
:1018F000252A309741F01092212A1092202A09952A
:101900008091202A089580E00895E091222AF091A4
:10191000232A309759F030911F2A20911E2A32171E
:1019200028F010921F2A80931E2A09940895089582
:10193000E0911F2A80911E2AE81730F4F0E0E25669
:10194000F64D808190E008958FEF9FEF089590917C
:101950001F2A80911E2A2FEF3FEF981748F4E92F96
:10196000F0E0E256F64D208130E09F5F90931F2A11
:10197000C901089580911E2A90911F2A891B990BF5
:101980000895CF92DF92EF92FF920F931F93CF9320
:10199000DF937C018A01EB016B01C40ED51ECC15CF
:1019A000DD0551F06991D701ED91FC910190F08135
:1019B000E02DC7010995F3CFC801DF91CF911F91A9
:1019C0000F91FF90EF90DF90CF9008952091202A03
:1019D00027FF08C021E030E0FC012283338390E040
:1019E00080E008958091212AE82FF0E0E25EF64D34
:1019F00060838F5F8093212A8093202A81E090E08A
:101A00000895DC01ED91FC91008CF18DE02D61E0F9
:101A100009940F938091372A9091382A0197A1F465
:101A20008091422A811112C0062F20E04091202A85
:101A30006EE179E280911D290E946E0B1092212A9D
:101A40001092202A0F91089580E0F8CF81E0F6CF20
:101A500060931D291092212A1092202A0895DC01FA
:101A6000ED91FC91048CF58DE02D21E009940F930C
:101A70008EE999E280932A2A90932B2A8091372A23
:101A80009091382A0197C9F48091422A811117C098
:101A9000FA014138510510F0E0E8F0E0022F862FFE
:101AA0002E2F40E070E060E00E946E0B10921F2A23
:101AB00080931E2A90E00F91089580E0F7CF81E097
:101AC000F5CFCB01BA010C94FE0BE0EAF8E01382EB
:101AD000168281E08583148611861092372A10922F
:101AE000382A089510921F2A10921E2A1092212A35
:101AF0001092202A8091372A9091382A892BD9F484
:101B000082E090E08093372A9093382A1092362A08
:101B10001092352A1092282A1092292A10921C29F4
:101B20001092332A660F6093AC0881EE8093A90867
:101B300081E08093A30885E79CE08093262A909318
:101B4000272A8EE199E280932C2A90932D2A85E80A
:101B50009CE08093312A9093322A8EE999E2809317
:101B60002E2A90932F2A80E88093302A089510928D
:101B70001F2A10921E2A1092212A1092202A809148
:101B8000372A9091382A892B41F562E070E086E18E
:101B90000E948F0562E070E087E10E948F058091CE
:101BA000E3058093E30581E090E08093372A9093EA
:101BB000382A10923B2A10923C2A1092422A109204
:101BC000412A81EC8093A30860EA76E881E090E006
:101BD0000E94FE0B81E08093A5080895CF93DF93C8
:101BE000EC018B818823D1F089819A81DC01ED9110
:101BF000FC910688F789E02D6881099589819A8191
:101C0000DC01ED91FC91028CF38DE02D099591E0C2
:101C1000811190E0892FDF91CF91089589819A8178
:101C2000DC01ED91FC910684F785E02D099581E0BA
:101C30008B83CE010E94EE0D982F8111D5CFEACF74
:101C4000FC01A5A1B6A18C9192A589238C93A5A195
:101C5000B6A18C9191A5892B8C930895DC01939664
:101C6000ED91FC919497908198968C918923808333
:101C70000895DC019396ED91FC919497908197964D
:101C80008C91892B80830895DC019196ED91FC91D4
:101C90009297908196968C91892380830895DC0198
:101CA0009196ED91FC919297908195968C91892BCC
:101CB00080830895CF92DF92EF92FF921F93CF938C
:101CC000DF93EC016A017B018DA981112BC08F2D5F
:101CD0009927AA27BB278093C4088091C30887FF50
:101CE000FCCFC701AA27BB278093C4088091C308F3
:101CF00087FFFCCFBB27AF2D9E2D8D2D8093C40871
:101D00008091C30887FFFCCFC092C4088091C308AC
:101D100087FFFCCFDF91CF911F91FF90EF90DF9075
:101D2000CF9008958130B1F410E2CE01F7FE0FC0DC
:101D30000E944F0ECE010E94390ECE010E942E0E3F
:101D4000CC0CDD1CEE1CFF1C115079F7E3CF0E9478
:101D5000440EF0CFEF8DF8A18F2D9927AA27BB272E
:101D60008083CE010E94200EEF8DF8A1C701AA2723
:101D7000BB278083CE010E94200EEF8DF8A1BB27E8
:101D8000AF2D9E2D8D2D8083CE010E94200EEF8DD4
:101D9000F8A1C082CE01DF91CF911F91FF90EF900B
:101DA000DF90CF900C94200EFF920F931F93CF9350
:101DB000DF93EC018B018DA9811112C01093C4082F
:101DC0008091C30887FFFCCF0093C4088091C308AB
:101DD00087FFFCCFDF91CF911F910F91FF90089566
:101DE0008130B1F490E1F92ECE0117FF0EC00E94B0
:101DF0004F0ECE010E94390ECE010E942E0E000F12
:101E0000111FFA94F110F0CFE5CF0E94440EF1CFEC
:101E1000EF8DF8A11083CE010E94200EEF8DF8A166
:101E20000083CE01DF91CF911F910F91FF900C9411
:101E3000200E0F931F93CF93DF93EC01162F8DA9E4
:101E400081110BC06093C4088091C30887FFFCCF49
:101E5000DF91CF911F910F910895813099F408E09F
:101E6000CE0117FF0CC00E944F0ECE010E94390E0A
:101E7000110FCE010E942E0E015091F7E9CF0E9462
:101E8000440EF3CFEF8DF8A16083CE01DF91CF91A7
:101E90001F910F910C94200ECF93DF93EC01ED8DE9
:101EA000FE8D80819CA989238083CE010E94190F19
:101EB000ED8DFE8D80819BA9892B8083DF91CF9151
:101EC00008958F929F92AF92BF92CF92DF92EF923E
:101ED000FF920F931F93CF93DF93EC0189AD9AADDF
:101EE000680F791F8BAD9CAD480F591F21503109E8
:101EF000260F371F4901B12CA12CCB01B0E0A0E087
:101F0000DC0199278827882A992AAA2ABB2A6801EE
:101F100081E0C81AD108C40ED51EF12CE12C70E066
:101F200060E0BA0155274427C42AD52AE62AF72AB1
:101F30006AE2CE010E944C0FB501A401CE010E94BD
:101F40005A0E6BE2CE010E944C0FB701A601CE01E2
:101F50000E945A0E6CE2CE01DF91CF911F910F913A
:101F6000FF90EF90DF90CF90BF90AF909F908F90B9
:101F70000C944C0FDC01D5962C91D59721110AC0F9
:101F80005F968D919C91DC01ED91FC910088F18927
:101F9000E02D099408950F931F93CF93DF93EC01E5
:101FA0002DA9211121C0DC018F8D98A1EC01E881C0
:101FB000F9810684F785E02D91960C919197929680
:101FC0001C91929793962C91939794963C91949709
:101FD00095964C91959796965C91969797966C915D
:101FE000979798967C910995DF91CF911F910F91CA
:101FF00008950F931F93CF93DF93EC018B010E9401
:10200000CB0F8FA987FD06C0EB8DFC8D80819AA92F
:1020100089238083ED8DFE8D80819CA98923808317
:1020200066E3CE010E94190FED8DFE8D80819BA984
:10203000892B80838DA9F8018230A1F06081CE01C7
:102040000E94190F8FA987FD06C0EB8DFC8D808142
:1020500099A9892B8083CE01DF91CF911F910F9198
:102060000C94BA0F88A9882349F360817181CE014D
:102070000E94D40EE7CFCF93DF931F92CDB7DEB788
:10208000FC0119826370668BDC01AD5BBF4F2C9144
:1020900030E011968C9190E0623031F06330C9F0FD
:1020A000613081F040EC498321AF32AF83AF94AF10
:1020B000BE016F5F7F4FCF010E94F90F0F90DF913C
:1020C000CF91089540EA498323AF34AF81AF92AFF7
:1020D000EFCF40E6F8CF0F931F93CF93DF931F927C
:1020E000CDB7DEB7FC0119826370668BDC01A85B9B
:1020F000BF4F2D913C91119712968D919C9162301A
:10210000D1F1633009F440C08F010C5B1F4F613087
:10211000F9F040EC4983AF014D5B5F4FDA014C9120
:1021200050E041AF52AFD8014C9150E043AF54AFB3
:102130002087318782879387BE016F5F7F4FCF01F2
:102140000E94F90F0F90DF91CF911F910F91089589
:1021500040EA4983D8014C9150E041AF52AFDF01D2
:10216000AA5BBF4F4C9150E043AF54AF22873387F7
:1021700080879187E1CFDF01AA5BBF4F4C9150E090
:1021800041AF52AF1196D0CF40E64983DF01A95B42
:10219000BF4F4C9150E041AF52AF1497E3CF1F9324
:1021A000CF93DF93EC01162FE881F9810284F38548
:1021B000E02D0995112371F06DADCE010E944C0FF9
:1021C000E881F9810688F789E02DCE01DF91CF9172
:1021D0001F9109946EADF1CFAF92BF92CF92DF9273
:1021E000EF92FF920F931F93CF93DF93EC0177FD54
:1021F00038C088859985681779079CF557FD31C0E7
:102200008A859B854817590764F569017A015B0146
:10221000E881F9810284F385E02DCE010995E881FA
:10222000F98102A4F3A5E02D01E010E021E030E007
:10223000A701B501CE010995B601CE010E94D40EC9
:10224000E881F9810688F789E02DCE01DF91CF91F1
:102250001F910F91FF90EF90DF90CF90BF90AF90C4
:102260000994DF91CF911F910F91FF90EF90DF9034
:10227000CF90BF90AF9008958F929F92AF92BF92F0
:10228000CF92DF92EF92FF920F931F93CF93DF9342
:10229000EC0149015701E881F98102A4F3A5E02D81
:1022A00009959401D8010E94C0556B017C01C114AD
:1022B000D104E104F10409F481C08DA9811119C090
:1022C00081E0C81AD108E108F1088FEFC816D806D6
:1022D000E806F80609F472C0B092C4088091C308F9
:1022E00087FFFCCFA092C4088091C30887FFFCCF72
:1022F000E7CF813099F581E0C81AD108E108F108EB
:102300008FEFC816D806E806F80609F457C00B2D5B
:1023100018E0CE0107FF1CC00E944F0ECE010E94A4
:10232000390ECE010E942E0E000F115091F70A2D8A
:1023300018E0CE0107FF0FC00E944F0ECE010E9491
:10234000390ECE010E942E0E000F115091F7D3CFFF
:102350000E94440EE3CF0E94440EF0CFBA1016C084
:10236000CC0CDD1CEE1CFF1CEF8DF8A1B08281E0CF
:10237000C81AD108E108F1088FEFC816D806E80698
:10238000F806E1F0CE010E94200EF1CF81E0C81ADC
:10239000D108E108F1088FEFC816D806E806F8065C
:1023A00069F0EF8DF8A1B082CE010E94200EEF8D72
:1023B000F8A1A082CE010E94200EE8CFDF91CF913C
:1023C0001F910F91FF90EF90DF90CF90BF90AF9053
:1023D0009F908F9008958F929F92AF92BF92CF92CD
:1023E000DF92EF92FF920F931F93CF93DF934C01F5
:1023F000EB016A01590137FF07C0C9010196C80FF7
:10240000D91FB194A194B108F401A085B185CA1770
:10241000DB070CF058C017FF07C0C8010196C80EB3
:10242000D91E119501951109F40182859385C8166D
:10243000D9060CF048C0FE01EA0DFB1DAF0141506A
:10244000510957FD40C0B601600F711F9B0121501B
:10245000310937FD38C0D7FF03C05F01D0E0C0E0CD
:10246000D7FE03C08B01D12CC12C4A175B071CF08F
:102470005D01AC1ABD0A281739071CF08C010C1934
:102480001D09D401ED91FC910284F385E02DC40176
:1024900009959501A601BE01C4010E943C11D40119
:1024A000ED91FC910688F789E02DC401DF91CF9171
:1024B0001F910F91FF90EF90DF90CF90BF90AF9062
:1024C0009F908F900994DF91CF911F910F91FF9072
:1024D000EF90DF90CF90BF90AF909F908F90089536
:1024E000EF92FF920F931F932115310529F00115EB
:1024F000110511F00E94EB111F910F91FF90EF90C9
:1025000008958F929F92AF92BF92CF92DF92EF92F7
:10251000FF920F931F93CF93DF935C014B016A01EE
:10252000E90177FD52C0DC0118968D919C916817E6
:1025300079070CF04AC0209709F447C037FF07C05D
:10254000C9010196C80ED91ED195C195D109F501D1
:1025500082859385C816D906C4F5A6014C0F5D1F68
:102560009A012150310937FD30C0D7FE03C0EA017E
:10257000D12CC12C281739071CF0EC01CC19DD092E
:10258000D501ED91FC910284F385E02DC5010995FB
:1025900078018E0121E030E0A601B401C5010E945E
:1025A0003C11D501ED91FC910688F789E02DC5011C
:1025B000DF91CF911F910F91FF90EF90DF90CF901F
:1025C000BF90AF909F908F900994DF91CF911F9112
:1025D0000F91FF90EF90DF90CF90BF90AF909F90C2
:1025E0008F9008958F929F92AF92BF92CF92DF9279
:1025F000EF92FF920F931F93CF93DF935C016B01D8
:102600004A01E90157FD52C0DC011A968D919C9157
:10261000481759070CF04AC0209709F447C037FF04
:1026200007C0C9010196C80ED91ED195C195D1091F
:10263000F50180859185C816D906C4F5A6014C0F11
:102640005D1F9A012150310937FD30C0D7FE03C00C
:10265000EA01D12CC12C281739071CF0EC01CC1948
:10266000DD09D501ED91FC910284F385E02DC501D2
:102670000995780101E010E09E01A401B601C501B1
:102680000E943C11D501ED91FC910688F789E02D5F
:10269000C501DF91CF911F910F91FF90EF90DF90D7
:1026A000CF90BF90AF909F908F900994DF91CF9182
:1026B0001F910F91FF90EF90DF90CF90BF90AF9060
:1026C0009F908F900895EF92FF920F931F93CF9357
:1026D000DF9377FD32C0DC011896ED91FC916E1707
:1026E0007F075CF52115310541F137FF07C0F9017E
:1026F00031964E0F5F1F319521953109DC011A96F5
:10270000ED91FC914E175F07C4F4EA01C20FD31F8D
:10271000DE011197B7FD11C057FF03C09E0150E0C5
:1027200040E0AE17BF071CF09F01241B350B78015A
:10273000890121E030E00E943C11DF91CF911F918F
:102740000F91FF90EF900895EF92FF920F931F93D8
:10275000CF93DF9357FD31C0DC011A96ED91FC91C8
:102760004E175F0754F52115310539F137FF07C0C2
:10277000F90131966E0F7F1F319521953109DC01EA
:102780001896ED91FC916E177F07BCF4EB01C20F18
:10279000D31FDE011197B7FD10C077FF03C09E0164
:1027A00070E060E0AE17BF071CF09F01261B370BDF
:1027B000780101E010E00E943C11DF91CF911F9160
:1027C0000F91FF90EF9008958F929F92AF92BF92DA
:1027D000CF92DF92EF92FF920F931F93CF93DF93ED
:1027E00047012115310509F44BC00115110509F404
:1027F00047C037FF07C0F90131966E0F7F1F319533
:1028000021953109DC011896AD90BC906A157B05C5
:10281000BCF517FF07C0F80131964E0F5F1F1195E9
:1028200001951109DC011A96ED91FC914E175F0795
:102830003CF56B01C20ED31EE6012197D7FD20C0E7
:102840007A01E00EF11ED7011197B7FD19C077FF8D
:1028500003C0960170E060E057FF03C0870150E0BD
:1028600040E0CA15DB051CF09501261B370BAE179F
:10287000BF071CF08F01041B150B74010E943C1153
:10288000DF91CF911F910F91FF90EF90DF90CF904C
:10289000BF90AF909F908F900895EF92FF920F930B
:1028A0001F93CF93DF93EC0177FD22C08885998534
:1028B00068177907ECF457FD1BC08A859B8548177C
:1028C0005907B4F47901E881F98102A4F3A5E02D58
:1028D00001E010E021E030E0CE010995B701CE0122
:1028E000DF91CF911F910F91FF90EF900C94D40E38
:1028F000DF91CF911F910F91FF90EF900895DC0130
:10290000D7962C91D79727FD09C05B96ED91FC9146
:102910005C972081D1963C91232B20830C94BA0F95
:10292000CF93DF93EC010E94CB0F8FA987FD06C0E8
:10293000EB8DFC8D80819AA989238083DF91CF91D3
:1029400008950895FC016370668B848195812681CA
:102950003781613039F0633029F080879187228791
:1029600033870895208731878287938708952F9230
:102970003F924F925F926F927F928F929F92AF920F
:10298000BF92CF92DF92EF92FF920F931F93CF935C
:10299000DF93CDB7DEB76A97CDBFDEBF898F9A8F41
:1029A00069837A834A01D22E0F8318873701BC2CA2
:1029B000DC0159962D913C915A972115310509F06A
:1029C00012C118968D919C911997681779070CF090
:1029D000D4C11A968D919C91481759070CF0CDC11E
:1029E0004C2C512CB6E0CB9E600D711D11246B87D1
:1029F0007C87161617060CF0C0C1EA2DF0E0E987B7
:102A0000FA8793E0EE0FFF1F9A95E1F7EF87F88BB7
:102A1000CF01840F951F181619060CF0AEC1A98DB1
:102A2000BA8D58968C91811104C0BFEABD1508F487
:102A3000D394A98DBA8DED91FC9111970284F38501
:102A4000E02DCD010995B5E0DB9EC0011124E9819F
:102A5000FA81EB83FC83312C212C9C0128513D4FC2
:102A60002F8B388F4A2D50E04D8B5E8BEF89F88D80
:102A7000E20DF31D44918D829E82D12CC12C69817F
:102A80007A81620D731D698B7A8B842F90E08B8B1A
:102A90009C8BE98DFA8DA081B18140FF7FC0F1E070
:102AA000BF126CC0AF126AC01C96ED91FC912F81D1
:102AB0003885A4014C0D5D1D69897A89898D9A8DAF
:102AC0000995EB89FC89F595E7954E2F5FEFC51ABF
:102AD000D50A6D817E818D899E89680F791F6D83EE
:102AE0007E8398E0C916D10481F6AFEF2A1A3A0A1C
:102AF000EB81FC81E40DF51DEB83FC83F5E02F16E3
:102B0000310409F0B3CF2F81388526153705B9F088
:102B1000A98DBA8DED91FC91B1E0BB1254C0AB12FE
:102B200052C069817A816B5F7F4F0088F189E02D07
:102B3000830128E030E0A401898D9A8D0995A98D43
:102B4000BA8DED91FC9111970688F789E02DCD01A2
:102B50006A96CDBFDEBFDF91CF911F910F91FF909D
:102B6000EF90DF90CF90BF90AF909F908F907F902D
:102B70006F905F904F903F902F9009941E96ED912B
:102B8000FC91EF80F88409851A8592014D815E8160
:102B90006B817C81898D9A8D099593CF2F813885A2
:102BA0002615370509F48DCF31E0B31207C0A31203
:102BB00005C01C96ED91FC9193017BCF1E96ED9183
:102BC000FC917301E0CF6B857C85641975090684DF
:102BD000F785E02D73010F8518899201A401898D75
:102BE0009A8D0995ACCFF90134969491329745911D
:102BF0005491D91AB7E0DB9E400D511D1124F90103
:102C0000259134912B8B3C8BFA0125903490FA015D
:102C10003296749031963491398B32966490319615
:102C2000449041E04C1518F04A1508F07FC0662D1D
:102C3000062C000C770B6B837C83842D042C000CFA
:102C4000990B8D839E83A98DBA8DED91FC9111977F
:102C50000284F385E02DCD010995512CD12CC12C96
:102C6000EA2DF0E0E987FA872B2D30E02B873C87AF
:102C7000A401440D511D47FC5A954F8B588F698113
:102C80007A81660D711D67FC7A956D877E877989DB
:102C9000C71608F054CF2C2D30E04D815E81420FD5
:102CA000531FA985BA854A9FC0014B9F900D5A9F1B
:102CB000900D1124FC01E80DF91DEF87F88B852D8F
:102CC000612C4F89588D420F531F4D8B5E8B6714BB
:102CD00008F050C044244394480E877041F4C10169
:102CE0000196EB89FC89E20DF31DD4901C01D7FEFF
:102CF00019C0A98DBA8DED91FC91662D70E0B1E0FF
:102D0000BB1219C0AB1217C02D853E85620F731F11
:102D10000484F585E02D2F8138854D895E89898D64
:102D20009A8D0995DD0C6394842DD1CF1D821E826E
:102D30001B821C8288CF4B815C81640F751FAB8521
:102D4000BC856A9FC0016B9F900D7A9F900D1124E6
:102D500069817A81680F791F0684F785E02DEF80FD
:102D6000F88409851A859D014F855889898D9A8D2A
:102D70000995D8CF570CC3948ACF6A96CDBFDEBFD2
:102D8000DF91CF911F910F91FF90EF90DF90CF9047
:102D9000BF90AF909F908F907F906F905F904F907B
:102DA0003F902F9008958F929F92AF92CF92EF9283
:102DB000FF920F931F93CF93DF93EC01262F898D02
:102DC0009A8D009709F051C06A30D1F41C861D8697
:102DD0008D8948E0849F900111248E859F85820F04
:102DE000931F8E879F8781E090E0DF91CF911F91A5
:102DF0000F91FF90EF90CF90AF909F908F9008959C
:102E00006D3089F3CC88AD888F898823C1F08C859B
:102E10009D8536E0C39E800D911D112448855985FE
:102E20004817590764F44E855F851C861D8638E077
:102E3000A39EC0011124840F951F8E879F87EA8867
:102E4000FB88088919894E855F856C857D85CE0153
:102E50000E94B7142C898C859D8546E0249F800DA7
:102E6000911D11248C879D87BECF6A3069F41C8622
:102E70001D86FC013896E4912D898E859F85E29F01
:102E8000800D911D1124ADCF6D3009F4ACCFFC0144
:102E900034963491631708F4A6CF3296E491E6177E
:102EA00008F4A1CFFC01329685909490462F431BE5
:102EB000342F47E0349F800C911C1124F40132968A
:102EC00034913196E4913323A9F1EE2399F1CC8822
:102ED000F4013596E491AD884F89442301F10E2E1B
:102EE000000CFF0BE30FF11DCE9EA001CF9E500DF5
:102EF00011246C857D85460F571F68857985641779
:102F000075076CF44E855F851C861D86FC0138961E
:102F1000E491AE9E400D511D11244E875F87EA88D3
:102F2000FB88088919894E855F856C857D85CE0172
:102F30000E94B714F4013496E4912C898C859D8508
:102F4000E29F800D911D11248DCF6F927F928F9201
:102F50009F92AF92BF92CF92DF92EF92FF920F9328
:102F60001F93CF93DF93EC016B015A0139014801A4
:102F7000E881F9810284F385E02D0995E881F981E2
:102F80000288F389E02D87019301A501B601CE01E6
:102F90000995A501480D591D41505109E881F98154
:102FA0000288F389E02D9301B601CE010995E881ED
:102FB000F9810088F189E02D9401A501B601CE01C7
:102FC0000995C60CD71CB60161507109E881F981D9
:102FD0000088F189E02D9401A501CE010995E881D1
:102FE000F9810688F789E02DCE01DF91CF911F91FD
:102FF0000F91FF90EF90DF90CF90BF90AF909F9098
:103000008F907F906F9009946F927F928F929F9292
:10301000AF92BF92CF92DF92EF92FF920F931F93E6
:10302000CF93DF935C01EB016A014901380187010D
:10303000DC01ED91FC916217730719F564167506B2
:103040002CF0962D872D3A01C92ED82E96012619DF
:1030500037092F5F3F4F048CF58DE02DA301BE0192
:10306000C5010995DF91CF911F910F91FF90EF90CE
:10307000DF90CF90BF90AF909F908F907F906F9098
:1030800008954615570591F42617370724F0892D22
:103090004B01C22FD82F9E01281939092F5F3F4FAE
:1030A000068CF78DE02DA601B401DACF0284F385FA
:1030B000E02D0995D501ED91FC910488F589E02D6D
:1030C00083019401A601BE01C5010995D501ED91C9
:1030D000FC910688F789E02DC501DF91CF911F9102
:1030E0000F91FF90EF90DF90CF90BF90AF909F90A7
:1030F0008F907F906F900994EF92FF920F931F93A0
:10310000DC011A960D911C911B9718962D913C91FC
:103110001997ED91FC9100A0F1A1E02D7B0150E009
:1031200040E070E060E009951F910F91FF90EF90F3
:1031300008954F925F926F927F928F929F92AF927B
:10314000BF92CF92DF92EF92FF920F931F93CF9394
:10315000DF936C012B015A0139014801DC01ED912B
:10316000FC910284F385E02D0995E201640C751C45
:10317000D601ED91FC91C615D7055CF40088F18964
:10318000E02D87019401A501BE01C6010995219694
:10319000EFCF0688F789E02DC601DF91CF911F910F
:1031A0000F91FF90EF90DF90CF90BF90AF909F90E6
:1031B0008F907F906F905F904F9009948F929F9225
:1031C000AF92BF92CF92DF92EF92FF920F931F9335
:1031D000CF93DF93EC015B014A016901E881F9813A
:1031E0000284F385E02D099595012C0D3D1D21509C
:1031F0003109E881F9810488F589E02D780184019D
:10320000A401B501CE010995E881F9810688F78905
:10321000E02DCE01DF91CF911F910F91FF90EF90A4
:10322000DF90CF90BF90AF909F908F9009948F9236
:103230009F92AF92BF92CF92DF92EF92FF920F9345
:103240001F93CF93DF93EC015B014A016901780181
:10325000E881F9810284F385E02D0995C80CD91C19
:10326000860101501109E881F9810488F589E02D72
:103270009501A401B501CE010995E881F98106887F
:10328000F789E02DCE01DF91CF911F910F91FF9033
:10329000EF90DF90CF90BF90AF909F908F90099468
:1032A000EF92FF920F931F93DC01ED91FC9100A030
:1032B000F1A1E02D09951F910F91FF90EF900895D6
:1032C0000F931F93DC01ED91FC91068CF78DE02D9F
:1032D00009951F910F9108950F931F93DC01ED91B4
:1032E000FC91048CF58DE02D09951F910F910895A7
:1032F000DC01ED91FC910084F185E02D09942F9281
:103300003F924F925F926F927F928F929F92AF9275
:10331000BF92CF92DF92EF92FF920F931F93CF93C2
:10332000DF93CDB7DEB72697CDBFDEBF3C016A0184
:103330002D833E83EB82FC825801A41AB50AB7FEA6
:1033400003C0B194A194B1088D809E80861A970A1B
:1033500097FE03C09194819491088A149B045CF0B9
:10336000902F812F0D811E819D838E839C2D8D2D0D
:103370006B01692F782F0C151D055CF09D818E81E6
:103380006D837E83692F782F902F812F8601C92E20
:10339000D82E1601201A310A2B012D813E81421AA6
:1033A000530A57FE03C0519441945108710137FEEE
:1033B00003C03FEFE31AF30AF594E7948D819E81F1
:1033C000861797075CF5A1E0B0E0A983BA83C01621
:1033D000D1064CF1D301ED91FC910484F585E02DEB
:1033E0002B813C81A8016D817E818A149B041CF095
:1033F0004D815E81B801C3010995E418F508F7FE17
:103400000AC02D813E8189819A81280F391F2D8321
:103410003E83E20CF31C0F5F1F4FD9CF2FEF3FEF1E
:1034200029833A83D4CF2696CDBFDEBFDF91CF91DB
:103430001F910F91FF90EF90DF90CF90BF90AF90D2
:103440009F908F907F906F905F904F903F902F90C4
:103450000895089590E080E00895DC01ED91FC91DD
:103460000088F189E02D23E030E00994CF92DF92CB
:10347000EF92FF920F931F93CF93DF93FC0127816D
:103480003085225031092230310530F58C010E94FF
:103490005D07F801C785D0890385148525853685A4
:1034A000601B710B820B930B9E010D2E000C440BC5
:1034B000550B0E942851AE01D7FF02C04F5F5F4FEE
:1034C000559547956A01550FEE08FF0821E0C6168D
:1034D000D706E806F90608F020E0822FDF91CF91A9
:1034E0001F910F91FF90EF90DF90CF900895862F5E
:1034F00090919F2A9923A1F06CE00E949A55E92FA0
:10350000F0E0EE0FFF1FE655F1418081918197FDBC
:1035100007C0809335289093362881E08093A12AB4
:103520000895FC012081318142815381FB0160813A
:103530007181828193810E9459510E943D52CB0139
:103540000895CF92DF92EF92FF920F931F93CF9344
:10355000DF936C019A018BE1869FE001879FD00D7C
:103560001124F12CE12C0BE110E0AE01B60184EC4A
:103570009DE20E947012E4ECFDE2C486D58623969B
:10358000C687D787DF91CF911F910F91FF90EF9062
:10359000DF90CF90089510920D2910920E2910926D
:1035A0000F29109210291092BD2A1092BE2A109253
:1035B00038281092392810923A2810923B281092FD
:1035C000092910920A2910920729109208290895B2
:1035D0004F925F926F927F928F929F92AF92BF9223
:1035E000CF92DF92EF92FF920F931F93CF93DF93CF
:1035F000CDB7DEB72E97CDBFDEBF80914528909125
:103600004628029709F04FC12091D12A298381E0F1
:1036100082278093C02A0E94FE064B015C013981FB
:10362000332309F438C18091A2289091A328A09156
:10363000A428B091A528A5019401281B390B4A0B99
:103640005B0BCA01B9010E94735269837A838B8331
:103650009C83209131283091322840913328509119
:1036600034280E94825320E030E044EB52E40E9470
:10367000CB5120E030E040E05FE30E945A510E94CD
:103680003D526B01770FEE08FF080091442C10911A
:10369000452CD8018C918E7F8C938C9186708230D2
:1036A00009F45FC0843051F081110FC044E0CC0CAC
:1036B000DD1CEE1CFF1C4A95D1F707C062E0F694B2
:1036C000E794D794C7946A95D1F780E090E0A1E0A1
:1036D000B0E08093522C9093532CA093542CB09331
:1036E000552C9701442755272B873C874D875E87AC
:1036F0002093462C3093472C4093482C5093492CD0
:10370000C701B6018827992760934A2C70934B2CE8
:1037100080934C2C90934D2C232B242B252B09F498
:1037200044C0412C512C32016394A30192012150D9
:103730003109410951092D833E834F8358876130F8
:10374000710581059105A9F4C701B6010E942851B0
:103750002B873C874D875E874D805E806F807884A5
:10376000E4CF53E0CC0CDD1CEE1CFF1C5A95D1F7C6
:10377000ACCF60934A2C70934B2C80934C2C90933D
:103780004D2C4092522C5092532C6092542C70929B
:10379000552C2B853C854D855E852093462C30939A
:1037A000472C4093482C5093492C8091522C909157
:1037B000532CA091542CB091552C0197A109B1091B
:1037C0008093522C9093532CA093542CB093552C4F
:1037D00040914A2C50914B2C60914C2C70914D2C67
:1037E000411551056105710561F0415051096109AB
:1037F000710940934A2C50934B2C60934C2C70933E
:103800004D2C4091462C5091472C6091482C709142
:10381000492C40934E2C50934F2C6093502C709316
:10382000512C452B462B472B21F480914A2C90910B
:103830004B2CD8011C968D939C931D971A961D9224
:103840001C921B978C9181608C93C501B4010E94DE
:1038500073526B017C0120E030E040EC5FE3698152
:103860007A818B819C810E9482539B01AC01C701AC
:10387000B6010E945A5120E030E04AE754E40E9429
:10388000CB510E9444526093CD2A7093CE2A8093EC
:10389000CF2A9093D02A8092A2289092A328A09217
:1038A000A428B092A5282E96CDBFDEBFDF91CF9180
:1038B0001F910F91FF90EF90DF90CF90BF90AF904E
:1038C0009F908F907F906F905F904F900895809120
:1038D000452890914628892B29F08091D12A882368
:1038E00009F454C08091462A9091472AA091482A11
:1038F000B091492A0196A11DB11D8093462A90934B
:10390000472AA093482AB093492A8091162890917B
:1039100017284091462A5091472A6091482A709171
:10392000492A092E000CAA0BBB0B481759076A0736
:103930007B0748F081E090E08093C32A9093C42AEB
:103940008093C12A0895809116289091172840915C
:10395000462A5091472A6091482A7091492A97FD3A
:10396000019695958795092E000CAA0BBB0B48175D
:1039700059076A077B0750F08091C32A9091C42AA7
:10398000892B21F01092C32A1092C42A08954F92D5
:103990005F926F927F928F929F92AF92BF92CF92DF
:1039A000DF92EF92FF92CF93DF93EC016A017B01EC
:1039B000488459846A847B848C809D80AE80BF80DB
:1039C00020E030E0A901C301B2010E94C651882362
:1039D000A1F1A5019401C701B6010E9459510E94AD
:1039E0003D529B0177FF04C022273327261B370B4C
:1039F000B901330F880B990B0E9475529B01AC01E2
:103A0000C301B2010E94C65187FF17C0CC82DD827C
:103A1000EE82FF826C817D818E819F81DF91CF91CB
:103A2000FF90EF90DF90CF90BF90AF909F908F90DE
:103A30007F906F905F904F900895488059806A8082
:103A40007B80A301920160E070E080E89FE30E9428
:103A50005951A50194010E9482534B015C01A701B9
:103A60009601C301B2010E9482539B01AC01C501C2
:103A7000B4010E945A516C837D838E839F83CACF89
:103A80008550883070F4E82FF0E0E75BF24E0C943C
:103A9000BA555C1D641D6C1D741D7C1D841D8C1D20
:103AA000941D60937E2870937F2864E47EE184E017
:103AB0000E94310481E008956093802870938128EA
:103AC0006EE37EE185E0F4CF6093822870938328D3
:103AD00068E37EE186E0ECCF6093842870938528CC
:103AE00062E37EE187E0E4CF6093862870938728C5
:103AF0006CE27EE188E0DCCF6093882870938928AF
:103B000066E27EE189E0D4CF60938A2870938B28A7
:103B100060E27EE18AE0CCCF60938C2870938D28A0
:103B20006AE17EE18BE0C4CF60938E2870938F288A
:103B300064E17EE18CE0BCCFDC01ED91FD91808100
:103B4000ED91FD919081ED91FD916C9163708E23CB
:103B500009F064609F2309F06860E9EBFDE1E60F7E
:103B6000F11D659565956D936D917D918D919D91FB
:103B7000099423C01AC012C016C010C01EC009C0CC
:103B800014C013C006C019C009C00DC007C00DC0C5
:103B900014C062507040804090400BC06150704033
:103BA0008040904006C06E5F01C06F5F7F4F8F4FB7
:103BB0009F4F9E938E937E936E9308958091A0283D
:103BC0009091A1280C949C1D80919E2890919F28F3
:103BD0000C949C1D80919C2890919D280C949C1D78
:103BE00080919A2890919B280C949C1D80919828F4
:103BF000909199280C949C1D8091962890919728DB
:103C00000C949C1D80919428909195280C949C1D57
:103C100080919228909193280C949C1D80919028DB
:103C2000909191280C949C1D80918E2890918F28C2
:103C30000C949C1D80918C2890918D280C949C1D37
:103C400080918A2890918B280C949C1D80918828C3
:103C5000909189280C949C1D8091862890918728AA
:103C60000C949C1D80918428909185280C949C1D17
:103C700080918228909183280C949C1D80918028AB
:103C8000909181280C949C1D80917E2890917F2892
:103C90000C949C1D80917C2890917D280C949C1DF7
:103CA00080917A2890917B280C949C1D8091782893
:103CB000909179280C949C1D80917628909177287A
:103CC0000C949C1DCF93DF93EC018B85823060F4C4
:103CD000F894CE010E949C1D6F81788589859A8514
:103CE0007894DF91CF910895F894F6CF0F931F93B6
:103CF000CF93DF93EC01062F142F70E060E0802F4C
:103D00000E945F0661E070E0802F0E945A0670E01A
:103D100060E0812F0E945F0661E070E0812F0E94C9
:103D20005A06802F90E0FC01E452F041A081A630B9
:103D300008F04EC020E2A29FD0011124BC5F9D017B
:103D4000285F3F4F288339838E539041FC01408187
:103D50004C83812F90E0FC01E452F041E08170E05F
:103D600060E0E63030F420E2E29FF0011124BF0170
:103D70007C5F9B01285F3F4F2A833B838E5390419A
:103D8000FC0130813D831F82188619861A868BE3D9
:103D90009FE10197F1F718962C91242381E009F413
:103DA00080E0FB019085932309F082608E83BE0141
:103DB000802F0E94401D8B87BE01812F0E94401DD5
:103DC0009B85890F8B87DF91CF911F910F9108956C
:103DD000B0E0A0E0B4CFCF93DF934091C12D21E0BC
:103DE00030E0D90102C0AA0FBB1F8A95E2F7CD01CE
:103DF0006230E1F4842B8093C12DC091C22DD0910B
:103E0000C32D8C819D81892BA1F089819A81DC0150
:103E1000ED91FC910688F789E02D6881099561ECA8
:103E20007DE2CE01DF91CF910C94600480958423D4
:103E3000E2CF80E0DF91CF910895CF93DF9340915F
:103E4000C12D21E030E0D90102C0AA0FBB1F8A9525
:103E5000E2F7CD016623E1F0842B8093C12DC09160
:103E6000C22DD091C32D8C819D81892BA1F0898198
:103E70009A81DC01ED91FC910688F789E02D68813B
:103E8000099561EC7DE2CE01DF91CF910C94600445
:103E900080958423E2CF80E0DF91CF9108958F92C7
:103EA0009F92AF92BF920F931F93CF93DF93CDB7A3
:103EB000DEB7A197CDBFDEBF19A2423008F44AE0B9
:103EC0008E010F5D1F4F842E912CB12CA12CA501CA
:103ED00094010E942851E62FB901CA01EA302CF55D
:103EE000E05DD801EE938D01232B242B252B79F750
:103EF00090E080E0109769F0FD0101900020E9F763
:103F00003197AF014A1B5B0BBD0184EC9DE20E941F
:103F10009C08A196CDBFDEBFDF91CF911F910F917D
:103F2000BF90AF909F908F900895E95CDACFCF92C9
:103F3000DF92EF92FF92CF93DF936B017C016DE2F2
:103F400084EC9DE20E94D316EC0166277727CB0113
:103F50006C197D098E099F094AE00E944F1F8C0F42
:103F60009D1FDF91CF91FF90EF90DF90CF9008954C
:103F7000BC01990F880B990B97FD0C94971F4AE091
:103F80000C944F1FEF92FF920F931F93CF93DF93E9
:103F90000097A9F0409147285091482860914928FE
:103FA00070914A284D3D55406105710544F02091BE
:103FB0000028309101282F3F3F4F09F450C0209135
:103FC000DD2D3091DE2D232B51F42091D22D309117
:103FD000D32D2A5F3F4F2093D22D3093D32D2FED39
:103FE00032E02093DD2D3093DE2D1816190624F5CE
:103FF000EC018091472890914828A0914928B091E0
:104000004A288D3D9540A105B10584F1E090132922
:10401000F09014290FE310E028E330E048E350E08B
:1040200066EB70E084EC9DE20E94EB118FEF9FEF56
:1040300080930028909301288091DD2D9091DE2DB2
:10404000892B49F08091D22D9091D32D06978093A2
:10405000D22D9093D32D1092DD2D1092DE2DDF9175
:10406000CF911F910F91FF90EF90089580910028BC
:10407000909101288C179D07F9F2E0901A29F09091
:104080001B290FE310E028E330E048E350E066EB43
:1040900070E084EC9DE20E94EB118CEB90E0809349
:1040A000D02D9093D12D8EE690E08093D22D9093D9
:1040B000D32DCE010E94B81FC0930028D0930128B1
:1040C000BBCFFF920F931F93CF93DF93F62E2091D8
:1040D000402830914128AC01421B530B2817390767
:1040E00014F59A018093402890934128E901219783
:1040F00080919D2A882329F070E060E080E10E9491
:10410000F20510E000E061E070E080E10C171D07AF
:1041100074F40E94F20570E060E080E10E94F20514
:104120000F5F1F4FF0CF9A01285F3F4FDBCF0E94F8
:10413000F2050E94FE066093992A70939A2A809352
:104140009B2A90939C2AC1E0C0939D2AFF2031F0C6
:1041500061E085E00E941D1FC0939E2A8091402847
:10416000909141280196DF91CF911F910F91FF907F
:104170000C94C21FCF93DF93EC014CE050E061E060
:1041800070E080EC90E00E94A11A1C161D062CF431
:10419000CE01DF91CF910C94B81FDF91CF9108959C
:1041A000009769F0FC0101900020E9F73197AF0119
:1041B000481B590BBC0184EC9DE20C949C0890E0D8
:1041C00080E00895CF93DF93873F2FEF920724F489
:1041D000DF91CF910C94B81FEC0197FF06C089E2E4
:1041E00090EF0E94D020CE01F3CF86E290EFCA304C
:1041F000D105BCF788E290EF209799F78BE290EF1A
:10420000DF91CF910C94D02040EA50E062E070E062
:1042100090E080E00E94A11A0E945D078091E72A49
:104220009091E82A8093E52A9093E62A86309105BA
:104230009CF483E390EF0E94D0208091E52A909136
:10424000E62A8630910510F5880F991FFC01EC5C79
:10425000F0418081918115C089309105A9F740EA2C
:1042600050E062E070E090E080E00E94A11A88E3F4
:1042700090EF0E94D0208091E42A811104C084E94B
:1042800090EF0C94D0208FE290EFFBCF08958F92A7
:104290009F92AF92BF92CF92DF92EF92FF920F93D5
:1042A0001F93CF93DF937C016B018A01241735079D
:1042B00010F030E020E0E901219740EF50E063E0AA
:1042C00070E08AE090E00E94A11AC7010E94D0200D
:1042D00099E1E92E9CEFF92E8091562A9091572A68
:1042E0000E94621E4B01940121703327232B11F58C
:1042F00094012E193F0912161306DCF16E157F0585
:10430000C9F08FEF9FEFC80FD91FD7FF35C0C00F7F
:10431000D11F44E650E063E070E080EA90E00E9444
:10432000A11AFE01EE0FFF1FEC0DFD1D8081918192
:104330000E94D02080915A2A90915B2A0E943109D4
:10434000E0915A2AF0915B2A808580FD10C082FF9F
:104350000EC0CE01DF91CF911F910F91FF90EF9092
:10436000DF90CF90BF90AF909F908F900895740191
:10437000B3CF81E090E0C7CFC017D10754F2C01B84
:10438000D10BC7CFCF92DF92EF92FF922091A72A55
:10439000211156C041110EC0C090A628D090A72868
:1043A000E090A828F090A928C616D706E806F906D6
:1043B00009F446C06B017C01C092A628D092A728C0
:1043C000E092A828F092A9284CE350E064E070E065
:1043D0008CE390E00E94A11A809145289091462894
:1043E000892B79F081EBC81684E0D806E104F1044A
:1043F00044F083E490EFFF90EF90DF90CF900C9427
:10440000D020F7FE17C0C701B6010E94971F20E019
:1044100030E040E85FE3609131287091322880916C
:104420003328909134280E94C651882349F085E4AE
:1044300090EFE1CF4AE0C701B6010E944F1FE7CFDE
:10444000FF90EF90DF90CF9008958F929F92AF9260
:10445000BF92CF92DF92EF92FF920F931F93CF9371
:10446000DF93962E7A01882361F040EA50E061E004
:1044700070E090E080E00E94A11A87E490EF0E9433
:10448000D02081E2C82E88E2D82ED0E0C0E09AE2A7
:10449000892E911051C0EC16FD0609F451C080918F
:1044A0000428909105288C179D0721F50FEF1FEF29
:1044B000F601A080B18063E070E0C430D10514F44F
:1044C00062E070E04AE250E0CE01837099279C01DF
:1044D000829EC001839E900D11240E94A11A009318
:1044E000D62D1093D72D0093D42D1093D52DC50123
:1044F0000E94E220219632E0C30ED11CC830D105C3
:1045000041F68FEF9FEF8093D62D9093D72D809318
:10451000D42D9093D52DE0920428F0920528DF91B8
:10452000CF911F910F91FF90EF90DF90CF90BF90B0
:10453000AF909F908F900895EC16FD0609F0B6CFCE
:1045400007EE19EFB5CF7F928F929F92AF92BF92F5
:10455000CF92DF92EF92FF920F931F93CF93DF934F
:10456000062F5A01882361F040EA50E061E070E0D4
:1045700090E080E00E94A11A82E590EF0E94D02096
:104580002FE6C22E2AE2D22ED0E0C0E010E03AE2BE
:10459000732E011169C0AC16BD0609F469C0809183
:1045A0000228909103288C179D0729F5EE24EA94A0
:1045B000FE2CF6018080918063E070E0C430D1056C
:1045C00014F462E070E04AE250E0CE018370992773
:1045D0009C01729EC001739E900D11240E94A11A2D
:1045E000E092D62DF092D72DE092D42DF092D52DD9
:1045F000C4010E94E220111107C011E0F601808180
:104600009181892B09F410E02196F2E0CF0ED11CA4
:10461000C830D10509F0BDCF8FEF9FEF8093D62D25
:104620009093D72D8093D42D9093D52D112341F0C5
:10463000809145289091462811E0892B09F410E0DB
:104640001093D12AA0920228B0920328DF91CF9133
:104650001F910F91FF90EF90DF90CF90BF90AF90A0
:104660009F908F907F900895AC16BD0609F09ECF65
:1046700087EEE82E89EFF82E9CCF1F93CF93DF9320
:10468000182F8091AE2AC6E0D0E081110AC0809137
:104690009F2AC0913C28D0913D28882311F0C7E083
:1046A000D0E08FEF9FEF8093D62D9093D72D8093FE
:1046B000D42D9093D52D82E08093D82D8093D92D41
:1046C00040EA50E0C930D10509F05DC062E070E019
:1046D00090E080E00E94A11A88E390EF0E94D02031
:1046E0008091E42A81114CC084E990EF0E94D0208F
:1046F00084EB90E08093D02D9093D12DCEE1D0E04B
:10470000C093D22DD093D32D8FE590EF0E94D0206F
:104710008CEC90E08093D02D9093D12DC093D22D2E
:10472000D093D32D81E690EF0E94D02080913E2837
:1047300090913F280E94BA201123D9F040EA50E01E
:1047400063E070E090E080E00E94A11A83E690EFC1
:104750000E94D02049E150E063E070E084E890E0FE
:104760000E94A11A8091832A9091842A01960E9426
:10477000B81F90E080E0DF91CF911F910C94C21F91
:104780008FE290EFB3CF61E070E090E080E00E94B4
:10479000A11ACC0FDD1FCC5CD04188819981A6CFB6
:1047A0008091F02C9091F12C0297029750F4809117
:1047B00060288823C9F150E040E061E081E00E9478
:1047C000A3228091DD2C9091DE2C0297029750F469
:1047D00080916128882389F150E040E061E081E028
:1047E0000E94252280916228882329F081E00E947E
:1047F0003D230E94042110925C2810925D281092A3
:104800005E2810925F2810926028109261288FEF26
:104810009FEF8093632890936428809365289093FA
:104820006628109262280895409165285091662864
:1048300057FDC7CF61E080E0C2CF4091632850911F
:10484000642857FDCFCF61E080E0CACFCF92DF92DE
:10485000EF92FF920F931F93CF93DF93EC010881A8
:1048600019816A817B81601B710B072E000C880BFC
:10487000990B0E9475529B01AC0160E070E080ECE6
:1048800091E40E94CB516B017C0168857985601BA6
:10489000710B072E000C880B990B0E9475529B011F
:1048A000AC01C701B6010E9482530E943F540E948E
:1048B0003D52CB0197FF02C00C96FCCF6CE070E03C
:1048C0000E94A655FC01EE0FFF1FE853F1418081C5
:1048D00091810197DF91CF911F910F91FF90EF9000
:1048E000DF90CF9008954F925F926F927F928F9258
:1048F0009F92AF92BF92CF92DF92EF92FF920F936F
:104900001F93CF93DF93CDB7DEB72E97CDBFDEBF1A
:10491000C0903128D0903228E0903328F09034288D
:10492000BC0104970CF0B2C06F5F7F4F072E000CE4
:10493000880B990B0E9475529B01AC0160E070E0FE
:1049400080E89FE30E94CB516093AA287093AB2824
:104950008093AC289093AD2820914528309146282B
:104960002230310561F421E02983A70196010E94DC
:10497000C651811101C0198239813093AE288090CF
:10498000AA289090AB28A090AC28B090AD2841E028
:104990004983A7019601C501B4010E94C651811146
:1049A00001C0198259815093582AA7019601C50167
:1049B000B4010E94C651882309F466C18091AE28D3
:1049C000811162C18092312890923228A0923328BE
:1049D000B092342860910A2870E090E080E00E9454
:1049E0007552A50194010E9482530E943D52AB0171
:1049F0008091112990911229BA010E94A6558093A5
:104A000011299093122980930B2990930C2960917E
:104A10004728709148288091492890914A280E94FF
:104A2000755269837A838B839C839B01AC0160EC14
:104A300071EE84E69CE40E94CB51A50194010E9492
:104A4000825320E030E044EB52E40E94CB510E94BC
:104A50003F540E9444526B017C010091442C109100
:104A6000452CD8018C918E7F8C938C9186708230EE
:104A700009F470C08430D9F0811120C044E0CC0C1E
:104A8000DD1CEE1CFF1C4A95D1F718C0635071095C
:104A9000072E000C880B990B0E9475526093AA2870
:104AA0007093AB288093AC289093AD2868CF62E0D8
:104AB000F694E794D794C7946A95D1F780E090E094
:104AC000A1E0B0E08093522C9093532CA093542CEF
:104AD000B093552C9701442755272B873C874D874A
:104AE0005E872093462C3093472C4093482C50935C
:104AF000492CC701B6018827992760934A2C7093E7
:104B00004B2C80934C2C90934D2C232B242B252B1A
:104B100009F444C0412C512C32016394A301920149
:104B200021503109410951092D833E834F83588714
:104B30006130710581059105A9F4C701B6010E9494
:104B400028512B873C874D875E874D805E806F8024
:104B50007884E4CF53E0CC0CDD1CEE1CFF1C5A958E
:104B6000D1F7ACCF60934A2C70934B2C80934C2C94
:104B700090934D2C4092522C5092532C6092542C76
:104B80007092552C2B853C854D855E852093462C57
:104B90003093472C4093482C5093492C8091522CB1
:104BA0009091532CA091542CB091552C0197A109B0
:104BB000B1098093522C9093532CA093542CB09312
:104BC000552C40914A2C50914B2C60914C2C70915B
:104BD0004D2C411551056105710561F04150510998
:104BE0006109710940934A2C50934B2C60934C2CD3
:104BF00070934D2C4091462C5091472C6091482C3D
:104C00007091492C40934E2C50934F2C6093502C14
:104C10007093512C452B462B472B21F480914A2C25
:104C200090914B2CD8011C968D939C931D971A96AE
:104C30001D921C921B978C9181608C9380914528CA
:104C400090914628892B01F5A501940169817A810B
:104C50008B819C810E94CB510E943D5240E02E9658
:104C6000CDBFDEBFDF91CF911F910F91FF90EF90ED
:104C7000DF90CF90BF90AF909F908F907F906F907C
:104C80005F904F900C94C2212E96CDBFDEBFDF9176
:104C9000CF911F910F91FF90EF90DF90CF90BF9039
:104CA000AF909F908F907F906F905F904F900895FE
:104CB0000F931F93CF93DF938091E72A9091E82A77
:104CC00088309105A9F440EA50E061E070E090E09E
:104CD00080E00E94A11A8EE690EF0E94D0201092F0
:104CE000402810924128DF91CF911F910F91089594
:104CF00010929F2A1092AE2A863091050CF04DC07A
:104D00008091E52A9091E62A80933C2890933D2853
:104D100082309105D1F481E08093422880E00E94A6
:104D20003D2380919F2A811104C08091AE2A88235F
:104D3000D1F240EA50E062E070E090E080E0DF9184
:104D4000CF911F910F910C94A11A049739F70CE39E
:104D500018E2C8E0D0E00E94E14FBE010E94A655D3
:104D6000D8015E962D913C915F97FC01EE0FFF1FDD
:104D7000E45BF74D808191815E968D939C935F9764
:104D8000332720833183219702501109209719F787
:104D90001092432810924428C1CF21E0873091051A
:104DA00009F020E020939F2A21E08630910509F048
:104DB00020E02093AE2A099709F0B0CF8091E42A31
:104DC00091E089278093E42A40EA50E062E070E0B5
:104DD00090E080E00E94A11A88E390EF0E94D0202A
:104DE0008091E42A81111AC084E990EF0E94D020BA
:104DF0008091452890914628892B61F08091E42A82
:104E0000882349F0209145283091462881E02130BF
:104E1000310509F080E08093D12A80CF8FE290EFB6
:104E2000E5CF20914528309146282230310509F000
:104E30004BC02091432A3091442A1216130624F4C1
:104E40008217130609F040C0842F90E024E0959566
:104E500087952A95E1F78770613161F0623129F118
:104E6000603191F590E0019680933E2890933F2821
:104E70000C94BA20863040F590E02091E72A3091DA
:104E8000E82A8217930701F18093E72A9093E82A92
:104E90008093E52A9093E62A8091582A882319F076
:104EA0001092582A08950C945826873069F0282FBC
:104EB00030E0843020F0C90103970C94732487E01C
:104EC00090E0821B930BF9CF0895CF93DF938091ED
:104ED0003C2890913D2882309105E1F150F4C09139
:104EE0003E28D0913F2821970197C1F0D0E0C0E043
:104EF00015C0C0914C28D0914D288430910571F097
:104F00000597A1F70E94E14F892F990F990B6091A6
:104F10003E2870913F280E94A655EC01109243282C
:104F20001092442860E0CE010E9461208091DD2C27
:104F30009091DE2C0197029788F4CC0FDD1FCF5D96
:104F4000D74D888199818093972A9093982ADF91F1
:104F5000CF91089581E080934228C8CF81E090E00E
:104F6000F2CF0F931F93CF93DF938091E42A88238E
:104F7000A9F088E790E0809316289093172881E0A5
:104F80008093452A80914B288823B1F181E080935A
:104F9000A02ADF91CF911F910F9108958091F02C5D
:104FA0009091F12C0197029768F7C0914028D09119
:104FB0004128CE01029608E010E0B8010E94A655F3
:104FC000FC01EE0FFF1FE159F54D20813181265A7A
:104FD0003F4FCE010196B8010E94A655FC01EE0F8D
:104FE000FF1FE159F54D80819181281B390B2093DA
:104FF000162830931728C6CFDF91CF911F910F91BC
:105000000C9465278091D12A811122C08091452876
:1050100090914628019721F48091BF2A81110AC0FE
:105020008091452890914628029771F48091C02A7A
:10503000882351F08091A02A882359F01092A02A49
:105040000E9465271092A12A1092BF2A1092C02AAE
:10505000089581E08093A12AF7CF0C9494560E9482
:105060001D57CF92DF92EF92FF920F93FC01C12C5C
:10507000B9E0DB2EBDE3EB2EF12CC082D182E282BF
:10508000F3821482158281E090E086839783C0903A
:105090001128D0901228E0901328F0901428F6944C
:1050A000E794D794C79490E04C155D056E057F0595
:1050B00040F4F694E794D794C7949F5F9630A1F795
:1050C00097E004600187892F8095A82FA170B0E038
:1050D00084E0AA0FBB1F8A95E1F791629A2B80E0CA
:1050E000232B09F480E4982B90870F91FF90EF9089
:1050F000DF90CF9008950F931F93CF93DF93CDB799
:10510000DEB72A97CDBFDEBF8C01FC0187818111FC
:105110000CC0108611861286138614861586168694
:105120001786108A118A81E087838091E305F80150
:105130009681892B8093E30561E070E083810E9472
:105140005F0661E070E0F80184810E945F06809153
:10515000C10884608093C1088091C00881628093F7
:10516000C00840915C2C50915D2C60915E2C709138
:105170005F2C0091602C2091622C3091632CCE0129
:1051800001960E94312899858A859093C008809362
:10519000C1082A96CDBFDEBFDF91CF911F910F913D
:1051A0000895CF92DF92EF92FF920F931F93CF93C8
:1051B000DF93EC016A017B01C114D104E104F10425
:1051C00039F4C12C88E4D82E88EEE82EFF24F3941D
:1051D000FE01FF96C082D182E282F38281E28DAF2E
:1051E00080E28EAF369610818FA987FD09C061E0FD
:1051F00070E00E945F0661E070E08FA90E945A068D
:1052000061E070E088AD0E945F0661E070E088AD0B
:105210000E945A068DA981114DC0C9A2DAA2EBA243
:10522000FCA2812F90E08DA39EA381E090E08FA34C
:1052300098A7812F90E0B0E0A0E089A79AA7ABA73C
:10524000BCA78F8D98A180579C4221F480E79CE2F7
:105250000E947B288EA987FD86C061E070E00E94D5
:105260005F0661E070E08EA90E945A0664E670E075
:1052700080E090E00E942D0770E060E08EA90E941F
:105280005A0664E670E080E090E00E942D0761E03D
:1052900070E08EA90E945A0668EC70E080E090E011
:1052A000DF91CF911F910F91FF90EF90DF90CF9002
:1052B0000C942D070CED1FEEF12C8130E1F461E030
:1052C00070E08AA50E945F0670E060E08AA50E94F7
:1052D0005A0661E070E08CA50E945F0670E060E015
:1052E0008CA50E945A068BA587FDB4CF70E060E0C4
:1052F0000E945F06AFCFF80181918F01863080F563
:10530000F0E28F9FC00111249C5F04962F8D38A17D
:105310002817390751F461E070E08F2D0E945F0675
:1053200070E060E08F2D0E945A06F39426E1F2129D
:10533000E2CF61E070E08EA50E945F0661E070E060
:105340008EA50E945A068FA587FD84CF61E070E08C
:105350000E945F0661E070E08FA50E945A067ACF36
:1053600090E080E0D2CFDF91CF911F910F91FF901D
:10537000EF90DF90CF9008955F926F927F928F921F
:105380009F92AF92BF92CF92DF92EF92FF920F93D4
:105390001F93CF93DF93CDB7DEB76297CDBFDEBF4C
:1053A0003C010B871C872D873E87042F4F87588B26
:1053B000698B7A8B29893A894B855C856D857E85D9
:1053C000CE0101960E94312859841A85D30118967E
:1053D0008C91882319F081FF18C0F8945092C0086E
:1053E0001093C1086296CDBFDEBFDF91CF911F91B0
:1053F0000F91FF90EF90DF90CF90BF90AF909F9074
:105400008F907F906F905F90089580FFE7CFF301BA
:1054100082849384A484B584C12CD12C7601B0E01D
:105420009401A501B601C701A0E00E94EC55A9F1C5
:10543000217030E040E050E060E070E080E090E01B
:105440000E94EC55E9F090E080E0B03370F48B2FCF
:10545000869586958695F0E28F9FC0011124805F26
:105460009B4F2B2F2770820F911DFC0140819301D0
:105470002B0F311DF901428BFC012081287F2083F5
:105480009401A501B601C70101E00E94D15549016F
:105490005A016B017C01BF5FC3CFD3011E968D9073
:1054A0009D90AD90BC905197C12CD12C7601B0E26B
:1054B0009401A501B601C701A0E00E94EC5509F4D2
:1054C0008DCF217030E040E050E060E070E080E09F
:1054D00090E00E94EC55E9F090E080E0B03370F489
:1054E0008B2F869586958695E0E28E9FC0011124CC
:1054F000805F9B4F2B2F2770820F911DFC014081F5
:1055000093012B0F311DF901428BFC012081287F73
:1055100020839401A501B601C70101E00E94D15585
:1055200049015A016B017C01BF5FC2CFFF920F930B
:105530001F93CF93DF938C01EB01F8800E9495506D
:10554000F81621F06F2DC8010E949D50CE01DF9109
:10555000CF911F910F91FF9008950F931F93CF93B9
:10556000DF938C01EB010E9495508883C80101965E
:105570000E9495508983CE01DF91CF911F910F91A9
:105580000895FF920F931F93CF93DF93EC018B014C
:10559000FB01F0800E949550F81621F06F2DCE018E
:1055A0000E949D50F801F1802196CE010E949550F5
:1055B000F81621F06F2DCE010E949D50C801DF9199
:1055C000CF911F910F91FF900895CF93DF93C0E18A
:1055D000D0E0BE016F5E774DCE010E94C12A2296B7
:1055E000C032D105B1F7DF91CF910895CF93DF930A
:1055F000C4E2D0E0BE01655B754DCE010E94C12AB8
:105600002296C433D105B1F7DF91CF910895CF939E
:10561000C62F80934B282AE530E02093162830933C
:10562000172861E0682784E00E941D1F60914B28C5
:1056300070E081E10E94F205CC2391F00E94B12735
:1056400080917F2A81110E94F62A8091802A8111FF
:105650000E94E52A1092802A10927F2ACF91089505
:105660008091E42A882361F388E790E080931628EC
:10567000909317281092452AE3CF90E00C94955010
:10568000882349F086E00E943D2B91E0811101C002
:1056900090E090931529809115292FE130E088231F
:1056A00011F020E038EF20931A2930931B2920EEC7
:1056B0003FEF882311F02FEF3FEF2093182930930D
:1056C0001929811107C08AE090E0809313299093F3
:1056D0001429089580E090EAF8CF6F927F928F921C
:1056E0009F92AF92BF92CF92DF92EF92FF920F9371
:1056F0001F93CF93DF93CDB7DEB7CA54D109CDBF87
:10570000DEBFD82E81E00E94402B1092A72A70E0C5
:1057100060E084EC9DE20E947C188091152861E095
:10572000811163E084EC9DE20E946B10E0901A29E5
:10573000F0901B290DE110E020EF30E050E040E058
:1057400070E060E084EC9DE20E94EB118FEF9FEF30
:105750008093D62D9093D72D8093D42D9093D52DD3
:105760008CE390E08093D02D9093D12D85E090E054
:105770008093D22D9093D32D82E08093D82D809367
:10578000D92D89E790EF0E94D020DD2009F413C2C3
:105790008AE090E08093D02D9093D12D8EE190E01F
:1057A0008093D22D9093D32D84E890EF0E94D02047
:1057B00068EE73E080E090E00E942D0780E1E8E46D
:1057C000FEEEDE01D39601900D928A95E1F7FE017F
:1057D000B39680E1DF011D928A95E9F77E01B3E37C
:1057E000EB0EF11C8F013F01470140E1C42ED12C8B
:1057F000BE016D5B7F4FC6010E94AD2A2596AEACFF
:10580000BFAC2597D401AD92BD924D01BE016F5F33
:105810007F4FC60144960E94AD2AB1E0AB1AB10891
:1058200049815A81E8E0AE16B10438F481E09A016A
:10583000245C3F4F2937310508F080E0D3014D93B8
:105840005D933D0181115AC084E00E943D2B91E09F
:10585000811101C090E09093372888E00E943D2B91
:1058600090E08093432A9093442A8AE00E943D2B43
:1058700091E0811101C090E09093622A8EE00E9435
:105880003D2B90E0809316299093172980915C2AF4
:1058900090915D2A0E94310980915A2A90915B2A49
:1058A0000E943109E0915A2AF0915B2A808580FD9F
:1058B000FEC140EF50E062E070E08AE090E00E94BC
:1058C000A11A89E890EF0E94D02080915C2A9091E3
:1058D0005D2ADC0118962C9120FF07C0E0915A2A1E
:1058E000F0915B2A208520FD29C00E94310980911A
:1058F0005A2A90915B2A0E943109E7CFE2E0CE0E4E
:10590000D11CF0E2CF16D10409F072CFA1E2B8E2C7
:105910004FE65AE2C7014096F701219131917F018C
:105920002D933D93F801219131918F01FA0121933B
:105930003193AF018E159F0579F786CF809158EE90
:10594000909159EEA0915AEEB0915BEE2B968CAFF0
:105950009DAFAEAFBFAF2B972091372881E02827AE
:1059600030E042E050E0BE01695B7F4F87E990EF95
:105970000E94472121E0892B09F020E0209337285D
:1059800067E378E284E090E00E94962A80915CEEE2
:1059900090915DEEA0915EEEB0915FEE27968CAF98
:1059A0009DAFAEAFBFAF27972091152930E042E001
:1059B00050E0BE016D5B7F4F84EA90EF0E9447216B
:1059C00021E0019709F020E02093152965E179E2B3
:1059D00086E090E00E94962A2091622A81E02827A2
:1059E00030E042E050E0BE01695B7F4F8CEA90EF0F
:1059F0000E94472121E0892B09F020E02093622AB0
:105A000062E67AE28AE090E00E94962A20911528C8
:105A100081E0282730E042E050E0BE01695B7F4F23
:105A200088EB90EF0E94472121E0892B09F020E0CC
:105A30002093152865E178E28CE090E00E94962A98
:105A4000209116293091172943E050E06BE078E26D
:105A500084EC90EF0E944721809316299093172998
:105A600066E179E28EE090E00E94C12A80911629D9
:105A70009091172963E070E00E94A655FC01EE0F9B
:105A8000FF1FEE53F141808180930A2882E2E0E615
:105A9000FEEEDE01119601900D928A95E1F72091BC
:105AA000432A3091442A41E150E0BE016F5F7F4FAD
:105AB0008AEC90EF0E9447218093432A9093442AD6
:105AC00063E47AE288E090E00E94C12A80E00E94CC
:105AD0006D2BBE016D5B7F4F90E080E00E94AD2A90
:105AE00025968EAD9FAD25971816190624F4809340
:105AF000082890930928BE016F5F7F4F82E090E0F5
:105B00000E94AD2A89819A811816190624F480937F
:105B100006289093072887E190E00E94F855FC0141
:105B20002091062830910728409108285091092893
:105B30008FEF9FEF8387948785879687838B948BDE
:105B400088E090E0858B968B40835183228333835A
:105B50001086118682E090E08483958384E190E052
:105B600086839783E093AC2AF093AD2AE091602A74
:105B7000F091612AF8941782108611861286789423
:105B8000E091562AF091572AF894178210861186D0
:105B90001286789487E090E08093542A9093552A57
:105BA0008091432A9091442A8093A72D9093A82D09
:105BB00080E00E94402B1092D02D1092D12D04E550
:105BC00010E00093D22D1093D32D83E091EF0E942B
:105BD000D0201092D02D1092D12D8FE690E080939E
:105BE000D22D9093D32D8FE091EF0E94D02080E0B2
:105BF0000E943D2380913E2890913F280E94BA2028
:105C000084E890E08093D02D9093D12D0093D22DF5
:105C10001093D32D88E090E00E94B81F8FEF9FEF84
:105C200080934528909346280E946E2FE0901A2971
:105C3000F0901B2903E410E02CE330E046E350E051
:105C400064EB70E084EC9DE20E94EB11E090182977
:105C5000F09019292CE330E046E350E064EB70E06B
:105C600084EC9DE20E94A517E0901829F090192974
:105C700001E410E02AE330E047E350E065EB70E038
:105C800084EC9DE20E94A517C65BDF4FCDBFDEBF4F
:105C9000DF91CF911F910F91FF90EF90DF90CF9008
:105CA000BF90AF909F908F907F906F900895E091FC
:105CB0005C2AF0915D2A808580FD0BCF40EF50E09B
:105CC00061E070E090E080E00E94A11A83ED90EF27
:105CD0000E94D02080915C2A90915D2AFC01208551
:105CE00020FF07C0E0915A2AF0915B2A208520FD11
:105CF00009C00E94310980915A2A90915B2A0E9422
:105D00003109E8CF1092D02D1092D12D89E3E82EE1
:105D1000F12CE092D22DF092D32D8DED90EF0E94D8
:105D2000D02060ED77E080E090E00E942D0784E1D4
:105D30000E94DC060FEF13E09801281B390B259613
:105D40002EAF3FAF259798E7C92ED12CC092D02D0A
:105D5000D092D12DE092D22DF092D32D85EE90EFFE
:105D60000E94D02025968EAD9FAD25970E94B81F2A
:105D70008AEE90EF0E94D02068EE73E080E090E021
:105D80000E942D071092D02D1092D12D24E5E22EE5
:105D9000F12CE092D22DF092D32D8CEE90EF0E9458
:105DA000D02060ED77E080E090E00E942D0784E154
:105DB0000E94DC06D801A81BB90BCD01A983BA83C8
:105DC000C092D02DD092D12DE092D22DF092D32D31
:105DD0000E94B81F25968EAD9FAD25978D599F4F78
:105DE00029813A8182179307DCF084E10E94DC0666
:105DF000F801E81BF90BE983FA8344E650E063E01D
:105E000070E088E790E00E94A11A89819A810E943F
:105E1000B81F64E670E080E090E00E942D07DACFC2
:105E200088E790E08093D02D9093D12D8FE690E07D
:105E30008093D22D9093D32D84EF90EF0E94D020A9
:105E40001092D02D1092D12D8AE890E08093D22D1F
:105E50009093D32D25968EAD9FAD25978438934092
:105E6000C4F589819A81883E93409CF587EF90EF35
:105E70000E94D02025968EAD9FAD2597809308284F
:105E80009093092889819A81809306289093072806
:105E900068E078E290E080E00E94C12A66E078E263
:105EA00082E090E00E94C12A68EB7BE080E090E015
:105EB0000E942D07F12CE12C07E810E020EF30E0E4
:105EC0004CE150E070E060E084EC9DE20E94EB1158
:105ED00000CE8CEF90EF0E94D020E6CFEF92FF92A1
:105EE0000F931F938FE00E94DC06893E23E0920708
:105EF00074F4833523E092070CF077C08536910562
:105F00000CF076C01F910F91FF90EF90089581E003
:105F100090E020914528309146282817390791F3C1
:105F2000809345289093462860E087E00E941D1FDB
:105F300070E060E080E10E94F205F12CE12C0BE1C1
:105F400010E028E730E04CE650E06CE370E084ECD1
:105F50009DE20E94EB1188E790E08093D02D909312
:105F6000D12D8FE690E08093D22D9093D32D809108
:105F70004528909146288130910509F45AC0D8F1FE
:105F8000029709F45BC00E94CB1A8091452890913A
:105F90004628892B61F08091E42A882349F02091DA
:105FA00045283091462881E02130310509F080E014
:105FB0008093D12A80913728882309F4A3CF0E94A7
:105FC0005D076093A82A7093A92A8093AA2A9093C8
:105FD000AB2A8091A72A882309F494CF80E01F91EF
:105FE0000F91FF90EF900C946D2B82E090E091CF99
:105FF00090E080E08ECF82E491EF0E94D02060910B
:106000004728709148288091492890914A280E94F9
:106010007552209131283091322840913328509187
:1060200034280E94CB510E943D5241E00E94C2217F
:10603000AACF87E491EF0E94D020A5CF8CE491EF06
:10604000FACF4F925F926F927F928F929F92AF9210
:10605000BF92CF92DF92EF92FF920F931F93CF9355
:10606000DF93CDB7DEB72E97CDBFDEBF8091452839
:1060700090914628019709F088C182E00E94350678
:1060800021E030E0892B11F030E020E02093C32A9A
:106090003093C42A82E00E943506019709F475C145
:1060A0002091D12A298381E082278093BF2A0E94F0
:1060B000FE064B015C013981332309F42EC1809126
:1060C0000D2990910E29A0910F29B0911029A501B9
:1060D0009401281B390B4A0B5B0BCA01B9010E94C2
:1060E000735269837A838B839C8320E030E044EB96
:1060F00052E40E94CB5120E030E040E05FE30E9498
:106100005A510E943D526B01770FEE08FF08009133
:10611000442C1091452CD8018C918E7F8C938C91BE
:106120008670823009F45FC0843051F081110FC055
:1061300044E0CC0CDD1CEE1CFF1C4A95D1F707C0D7
:1061400062E0F694E794D794C7946A95D1F780E01B
:1061500090E0A1E0B0E08093522C9093532CA09358
:10616000542CB093552C9701442755272B873C87F7
:106170004D875E872093462C3093472C4093482CC4
:106180005093492CC701B6018827992760934A2C60
:1061900070934B2C80934C2C90934D2C232B242BC1
:1061A000252B09F444C0412C512C32016394A301E6
:1061B000920121503109410951092D833E834F83BA
:1061C00058876130710581059105A9F4C701B601B1
:1061D0000E9428512B873C874D875E874D805E80CB
:1061E0006F807884E4CF53E0CC0CDD1CEE1CFF1CE8
:1061F0005A95D1F7ACCF60934A2C70934B2C809377
:106200004C2C90934D2C4092522C5092532C6092D7
:10621000542C7092552C2B853C854D855E852093A2
:10622000462C3093472C4093482C5093492C809116
:10623000522C9091532CA091542CB091552C019735
:10624000A109B1098093522C9093532CA093542C04
:10625000B093552C40914A2C50914B2C60914C2C72
:1062600070914D2C411551056105710561F041504A
:1062700051096109710940934A2C50934B2C60934A
:106280004C2C70934D2C4091462C5091472C609192
:10629000482C7091492C40934E2C50934F2C609376
:1062A000502C7093512C452B462B472B21F4809179
:1062B0004A2C90914B2CD8011C968D939C931D9742
:1062C0001A961D921C921B978C9181608C93C5012C
:1062D000B4010E9473526B017C0120E030E040EC7D
:1062E0005FE369817A818B819C810E9482539B014B
:1062F000AC01C701B6010E945A5120E030E04AE7E4
:1063000054E40E94CB510E9444526093CD2A709372
:10631000CE2A8093CF2A9093D02A80920D299092F2
:106320000E29A0920F29B09210298091AE2A8111D6
:1063300004C08091BF2A882341F1809137288823A7
:1063400021F10E945D076093A82A7093A92A809387
:10635000AA2A9093AB2A8091A72A8823B1F080E0E3
:106360002E96CDBFDEBFDF91CF911F910F91FF9091
:10637000EF90DF90CF90BF90AF909F908F907F90E5
:106380006F905F904F900C946D2B2E96CDBFDEBF1B
:10639000DF91CF911F910F91FF90EF90DF90CF9001
:1063A000BF90AF909F908F907F906F905F904F9035
:1063B00008950E945D076093A32A7093A42A809396
:1063C000A52A9093A62A8091852A9091862A63E037
:1063D00070E00E94A655892B01F564EF71E080E022
:1063E00090E00E942D0770E060E084EC9DE20E9446
:1063F0007C1864EF71E080E090E00E942D070E941D
:106400003D5023E030E040E050E00E94C5506E5F18
:106410007F4F6093192870931A280E943D5023E003
:1064200030E040E050E00E94C5506093952A7093A0
:10643000962A0E943D5022E330E040E050E00E9466
:10644000C550FB014091872A5091882A411551057A
:1064500009F47CC04330510509F478C02091CC2D5B
:106460003091CD2D261B370B2093892A30938A2A11
:106470004230510534F0E091CE2DF091CF2DE61B46
:10648000F70BE0938B2AF0938C2A2091CC2D30913E
:10649000CD2D4230510514F430E020E02093932AB2
:1064A0003093942A4115510529F030E020E0433023
:1064B000510521F42091CE2D3091CF2D20938F2A9C
:1064C0003093902A2091CC2D3091CD2D4230510522
:1064D00014F030E020E02093912A3093922A411565
:1064E000510539F04330510599F14091CE2D50912D
:1064F000CF2D40938D2A50938E2A0E943D502DE738
:1065000030E040E050E00E94C550675E7F4F8F4F03
:106510009F4F0E94755220E030E048E452E40E9410
:10652000CB5160931D2870931E2880931F28909351
:1065300020280E943D502FEF3FEF40E050E00E94A6
:10654000C55060931B2870931C2808959B018CCF25
:1065500050E040E0CECF3F924F925F926F927F9299
:106560008F929F92AF92BF92CF92DF92EF92FF9263
:106570000F931F93CF93DF93CDB7DEB72A97CDBF8D
:10658000DEBF8091452890914628029709F059C3B3
:106590004423F9F08091452890914628029709F00C
:1065A00050C360E080E02A96CDBFDEBFDF91CF917F
:1065B0001F910F91FF90EF90DF90CF90BF90AF9021
:1065C0009F908F907F906F905F904F903F900C9432
:1065D000072B662369F18091452890914628029700
:1065E00009F02FC30E94CB1A8FEF9FEF80931129E0
:1065F0009093122980930B2990930C2961E081E0FC
:106600000E94072B2A96CDBFDEBFDF91CF911F914D
:106610000F91FF90EF90DF90CF90BF90AF909F9041
:106620008F907F906F905F904F903F900C94E81AFE
:10663000222389F08091452890914628029709F0FD
:1066400000C30E94CB1A8FEF9FEF80931129909384
:10665000122960E0D4CF80911129909112290196DE
:10666000809311299093122980910B2990910C29E4
:10667000019680930B2990930C2920910929309140
:106680000A292F5F3F4F29873A87209309293093A2
:106690000A290E94FE066B017C0180900D299090D2
:1066A0000E29A0900F29B090102981149104A10403
:1066B000B10409F4BDC08C149D04AE04BF0408F0FD
:1066C000B7C0409038285090392860903A28709090
:1066D0003B2860910A2870E090E080E00E947552AB
:1066E000209131283091322840913328509134281C
:1066F0000E9482539B01AC0160E070E68AE697E459
:106700000E94CB5169837A838B839C83C701B60136
:106710000E9473526D837E838F839887C501B40175
:106720000E9473529B01AC016D817E818F8198859F
:106730000E9459519B01AC0169817A818B819C81B6
:106740000E94CB5120E030E04AE754E40E9482539B
:106750004B015C018091072990910829FC01EE0F03
:10676000FF1FEE0FFF1FE552F74D80829182A2823C
:10677000B38201966BE070E00E94A65580930729D2
:106780009093082989859A850B971CF18CE2EBED93
:10679000F8E2AFEAB8E201900D928A95E1F721E9BB
:1067A0003AE144E050E06BE070E08FEA98E20E944A
:1067B000284E8091C3289091C428A091C528B091FB
:1067C000C6288093382890933928A0933A28B0930C
:1067D0003B28A3019201609138287091392880915B
:1067E0003A2890913B280E9459510E943D529B01AA
:1067F00077FF04C022273327261B370BB901330F3D
:10680000880B990B0E947552A30192010E94CB51F3
:1068100020E030E040E85EE30E947D53181644F427
:106820008092382890923928A0923A28B0923B283A
:10683000C0920D29D0920E29E0920F29F0921029D2
:10684000409038285090392860903A2870903B2822
:10685000B301A2018AEC9CE20E94C71C0E943F5433
:1068600069837A838B839C8300910A2810E0B801A6
:10687000012E000C880B990B0E9475526B017C0154
:10688000209131283091322840913328509134287A
:106890000E9482530E943F540E943D526D837E832A
:1068A0002091E42A222319F13090452A072E000C6A
:1068B000880B990B0E9475524B015C018D819E8162
:1068C00063E070E00E94A655072E000C880B990B20
:1068D0000E9475529B01AC01C501B401332009F43B
:1068E0009CC00E945A510E943D526D837E838091CC
:1068F000112990911229ED81FE818E179F0709F0D1
:10690000B5C18091452A91E089278093452A10924C
:106910001129109212298091AE28882309F44BC1C5
:1069200080910B2990910C29B8010E94A655892BC2
:1069300009F041C11092AE2810920B2910920C2937
:106940008090AA289090AB28A090AC28B090AD2859
:106950008092312890923228A0923328B092342825
:106960008091452890914628029709F059C0A701C7
:106970009601C301B2010E94825320E030E040EC56
:1069800051E40E94CB510E943F540E943D5240E08E
:106990000E94C2216091472870914828809149281F
:1069A00090914A280E9475529B01AC0160EC71EEF7
:1069B00084E69CE40E94CB5120913128309132280A
:1069C00040913328509134280E94825320E030E0D7
:1069D00044EB52E40E94CB510E943F540E94445227
:1069E0006B017C012091442C3091452C2D833E83FA
:1069F000F90180818E7F808380818670823009F4E6
:106A00006DC0843019F1811128C0A4E0CC0CDD1CCC
:106A1000EE1CFF1CAA95D1F720C00E94595163CFEC
:106A20008091452890914628892B09F0B3CF609139
:106A30004728709148288091492890914A280E94BF
:106A40007552A50194010E94CB519FCF12E0F6949C
:106A5000E794D794C7941A95D1F780E090E0A1E02D
:106A6000B0E08093522C9093532CA093542CB0936D
:106A7000552C9701442755272093462C3093472CBB
:106A80004093482C5093492CC701B6018827992779
:106A900060934A2C70934B2C80934C2C90934D2CEC
:106AA0002115310541055105C9F1412C512C320107
:106AB000639453014201F1E08F1A9108A108B108D3
:106AC000613071058105910589F4C701B601A50101
:106AD00094010E94285124013501EBCFB3E0CC0C86
:106AE000DD1CEE1CFF1CBA95D1F7B7CF60934A2C82
:106AF00070934B2C80934C2C90934D2C4092522CA5
:106B00005092532C6092542C7092552C2093462C0A
:106B10003093472C4093482C5093492C8091522C11
:106B20009091532CA091542CB091552C0197A10910
:106B3000B1098093522C9093532CA093542CB09372
:106B4000552C40914A2C50914B2C60914C2C7091BB
:106B50004D2C411551056105710561F041505109F8
:106B60006109710940934A2C50934B2C60934C2C33
:106B700070934D2C4091462C5091472C6091482C9D
:106B80007091492C40934E2C50934F2C6093502C75
:106B90007093512C452B462B472B21F480914A2C86
:106BA00090914B2CED81FE81848795871286138608
:106BB00080818160808380910D2990910E29A09120
:106BC0000F29B0911029892B8A2B8B2B79F16981A0
:106BD0007A818B819C810E943D526B017C01809166
:106BE000BD2A9091BE2A092E000CAA0BBB0BC81619
:106BF000D906EA06FB06D1F0A0910A28B0E0A70169
:106C000096010E94E45028E130E040E050E00E940C
:106C1000C550CA01B9010E9475520E943D5240E020
:106C20000E94C221C092BD2AD092BE2A80914B28D8
:106C300081110E94E81A81E090E08093C32A90932A
:106C4000C42A2A96CDBFDEBFDF91CF911F910F914D
:106C5000FF90EF90DF90CF90BF90AF909F908F907C
:106C60007F906F905F904F903F9008952D813E816F
:106C700037FF04C02F5F3F4F2D833E83ED81FE81A0
:106C8000F595E795E817F907E4F61092C32A1092F4
:106C9000C42AD7CF1F920F920FB60F9211242F93B1
:106CA0003F934F935F936F937F938F939F93AF9394
:106CB000BF934091D82A5091D92A6091DA2A7091D5
:106CC000DB2A8091D62A9091D72A2091D42A30911C
:106CD000D52A420F531F611D711D2091D22A309178
:106CE000D32A820F931F883E23E0920730F0885EFC
:106CF00093404F5F5F4F6F4F7F4F8093D62A9093A3
:106D0000D72A4093D82A5093D92A6093DA2A7093CD
:106D1000DB2A8091E02A9091E12AA091E22AB091A9
:106D2000E32A0196A11DB11D8093E02A9093E12AE8
:106D3000A093E22AB093E32A81E08093B60ABF9140
:106D4000AF919F918F917F916F915F914F913F9103
:106D50002F910F900FBE0F901F9018951F920F92BA
:106D60000FB60F9211242F933F934F935F936F931E
:106D70007F938F939F93AF93BF93EF93FF9385E0A0
:106D80000E94C908FF91EF91BF91AF919F918F91A0
:106D90007F916F915F914F913F912F910F900FBE17
:106DA0000F901F9018951F920F920FB60F921124FB
:106DB0002F933F934F935F936F937F938F939F9303
:106DC000AF93BF93EF93FF9384E00E94C908FF91B4
:106DD000EF91BF91AF919F918F917F916F915F9153
:106DE0004F913F912F910F900FBE0F901F901895CC
:106DF0001F920F920FB60F9211242F933F934F9330
:106E00005F936F937F938F939F93AF93BF93EF9312
:106E1000FF9383E00E94C908FF91EF91BF91AF916A
:106E20009F918F917F916F915F914F913F912F91A2
:106E30000F900FBE0F901F9018951F920F920FB6D4
:106E40000F9211242F933F934F935F936F937F93F0
:106E50008F939F93AF93BF93EF93FF9382E00E9432
:106E6000C908FF91EF91BF91AF919F918F917F9151
:106E70006F915F914F913F912F910F900FBE0F90A7
:106E80001F9018951F920F920FB60F9211242F93F7
:106E90003F934F935F936F937F938F939F93AF93A2
:106EA000BF93EF93FF9381E00E94C908FF91EF9198
:106EB000BF91AF919F918F917F916F915F914F9112
:106EC0003F912F910F900FBE0F901F9018951F921A
:106ED0000F920FB60F9211242F933F934F935F930E
:106EE0006F937F938F939F93AF93BF93EF93FF9392
:106EF00080E00E94C908FF91EF91BF91AF919F91EF
:106F00008F917F916F915F914F913F912F910F9052
:106F10000FBE0F901F9018951F920F920FB60F92F1
:106F200011242F933F934F935F936F937F938F938E
:106F30009F93AF93BF93EF93FF9380E09DE20E94F6
:106F4000D704FF91EF91BF91AF919F918F917F9166
:106F50006F915F914F913F912F910F900FBE0F90C6
:106F60001F9018951F920F920FB60F9211242F9316
:106F70003F934F935F936F937F938F939F93AF93C1
:106F8000BF93EF93FF9380E09DE20E940209FF917F
:106F9000EF91BF91AF919F918F917F916F915F9191
:106FA0004F913F912F910F900FBE0F901F9018950A
:106FB0001F920F920FB60F9211242F933F934F936E
:106FC0005F936F937F938F939F93AF93BF93EF9351
:106FD000FF9389EA9BE20E94D704FF91EF91BF9152
:106FE000AF919F918F917F916F915F914F913F9161
:106FF0002F910F900FBE0F901F9018951F920F9218
:107000000FB60F9211242F933F934F935F936F937B
:107010007F938F939F93AF93BF93EF93FF9389EAEF
:107020009BE20E940209FF91EF91BF91AF919F9166
:107030008F917F916F915F914F913F912F910F9021
:107040000FBE0F901F9018951F920F920FB60F92C0
:1070500011242F933F934F935F936F937F938F935D
:107060009F93AF93BF93EF93FF9380914E2C90919A
:107070004F2CA091502CB091512C0197A109B1092E
:1070800080934E2C90934F2CA093502CB093512C66
:10709000181619061A061B063CF1892B8A2B8B2B16
:1070A000B9F18091462C9091472CA091482CB09139
:1070B000492C0097A105B10591F080934E2C909337
:1070C0004F2CA093502CB093512CE091442CF09174
:1070D000452C8091522C9091532C84879587E09178
:1070E000562CF091572C099581E08093A60AFF91C8
:1070F000EF91BF91AF919F918F917F916F915F9130
:107100004F913F912F910F900FBE0F901F901895A8
:1071100040914A2C50914B2C60914C2C70914D2CED
:107120004115510561057105A9F0E091442CF091DC
:10713000452C4487558782859385B0E0A0E084176D
:107140009507A607B70784F28091522C9091532C93
:10715000848795878091462C9091472CA091482C4C
:10716000B091492C80934E2C90934F2CA093502C8F
:10717000B093512CB4CF1F920F920FB60F921124DF
:107180002F933F934F935F936F937F938F939F932F
:10719000AF93BF93CF93EF93FF93C091AB08C2FF20
:1071A0000AC01092362A1092352A1092342A84E0AE
:1071B0000E94CB0B14C0C6FF2FC08091332A8130B0
:1071C00051F48091362AE091312AF091322A90E0F0
:1071D00009951092332AC0FF14C00E94DB0BFF9167
:1071E000EF91CF91BF91AF919F918F917F916F91CF
:1071F0005F914F913F912F910F900FBE0F901F9075
:10720000189580E48093AB0881E00E94CB0B8091BD
:10721000AB0885FFE4CFE1CFC7FF5CC0C3FF08C068
:107220001092362A1092352A1092342A83E0C0CF69
:107230008091A90880668093A9088091AB0881FF9E
:107240002CC08091352A882349F08091AB0884FFB7
:1072500005C082E08093AA0881E0AACF9091352AE8
:107260008091342A9817A8F4E091352A80912C2A2D
:1072700090912D2AE80FF92FF11D80818093AD08A0
:107280008091352A8F5F8093352A83E08093AA0806
:10729000A6CF82E08093AA088BCF9091362A809166
:1072A000302A981790F48091AD08E091362A209109
:1072B0002E2A30912F2AE20FF32FF11D8083809127
:1072C000362A8F5F8093362AE0CF86E08093AA0823
:1072D00082E06ECF85E06CCF1F920F920FB60F92B7
:1072E00011242F933F938F939F93EF93FF9380915C
:1072F000A508982F9C70E1F08091A50894E082FF8A
:1073000093E09093412A8093A50881E090E08093D8
:10731000372A9093382A1092422AFF91EF919F9139
:107320008F913F912F910F900FBE0F901F90189546
:1073300086FF4EC020913E2A90913D2A8091A5085B
:1073400084FF15C080913A2A882379F083E08093E6
:10735000A40885E08093412A1092422A81E090E0BF
:107360008093372A9093382AD8CF81E0F0CF80914C
:107370003C2A821790F4E0913C2A80913F2A909118
:10738000402AE80FF92FF11D80818093A808809191
:107390003C2A8F5F80933C2AC0CF80913B2A89177B
:1073A00060F484E090E08093372A9093382A8091AB
:1073B000392A81608093A708B0CF80913A2A882328
:1073C00029F083E08093A40881E0C4CF81E0FACF64
:1073D00087FF40C090913B2A80913D2A9817D8F4AE
:1073E0008091A808E0913B2A20912A2A30912B2AEB
:1073F000E20FF32FF11D808380913B2A8F5F8093F2
:107400003B2A90913D2A80913B2A8917D8F482E04B
:107410008093A40882CF80913A2A882389F087E05C
:107420008093A40882E08093412A1092422A81E04E
:1074300090E08093372A9093382A10923D2A6DCF9E
:1074400085E0EECF80913A2A882311F087E0BACF09
:1074500085E0B8CF86E07ECFEF92FF920F931F9327
:10746000CF93DF93A0E0BDE212961D921C9213977A
:1074700048EE53E060E070E014964D935D936D9399
:107480007C93179726E63FEE2D933C93119780E26D
:1074900098E01C968D939C931D971E961C921E97A8
:1074A00081E01F968C931F9794E050969C93509781
:1074B00052961C92529753961C92539754961C9234
:1074C000549755961C9255979BE156969C935697C8
:1074D00057961C92579758961C9258971092992D30
:1074E00010929A2DE9EAFBE21282138244835583BB
:1074F000668377832083318320E638E024873587CD
:1075000098E1968799E1978790E4908B128A138A85
:10751000148A158A96E2968B178A108E1092422C46
:107520001092432CE4E4FCE220E83AE0208331832B
:1075300012821382148215820AE010E020E030E00B
:107540000683178320873187128613861486158653
:107550000FEF1FEF20E030E006871787208B318B7D
:10756000ECE5FCE200E019E02DE330E0008311835C
:10757000228333831482158221E030E0268337830F
:10758000C0E7DCE2E0E8FFEEE883F9831F8212E067
:107590001E839CE09A839DE09C839BE09B8398E004
:1075A0009D83E4E6FCE21282138244835583668362
:1075B00077834EE95FEE40835183E4ECFDE2128273
:1075C000138260EF70E06483758340E451E046838A
:1075D00057836087718742875387168A148615867A
:1075E00016861786858B848B4FEF5FEF428B538B0C
:1075F000408B518B878B108E118E128E15AA89E0CD
:1076000086AB8AE087AB90AF11AE12AE13AE14AE6C
:1076100015AE16AE1092032E1092042E1092052E67
:107620001092062EC78FD0A344E854E0458F568FA2
:1076300093AB84E294E0838F948F11AB8DEF82AB98
:1076400087EF84AB1092072E1092082E1092092E0D
:107650008AEF9FEE8083918310920A2E10920B2E58
:10766000E0ECFDE210821182EBE9FDE2A083B18340
:1076700012821382148215822487358726873787E2
:107680000E945D076093FC2C7093FD2C8093FE2C70
:107690009093FF2C0E945D07C9EEDCE218821982EC
:1076A0001A821B821C821D821E821F8218861986E6
:1076B0001A860E945D076B877C878D879E878CE288
:1076C000E82EFF24F394EF86F88A04E110E0098B9A
:1076D0001A8BC6EDDCE2188219821A821B821C8288
:1076E0001D821E821F82188619861A860E945D07D7
:1076F0006B877C878D879E87EF86F88A098B1A8B2C
:10770000EAECFCE28AE999E9A9E1BEE3808391838E
:10771000A283B38380E090E0A0EFB2E484839583FA
:10772000A683B783EEEBFCE24DEC5CEC6CE47DE30E
:10773000408351836283738340E050E060E074E4EF
:107740004483558366837783E2EBFCE24AE959E997
:1077500069E97EE3408351836283738384839583E5
:10776000A683B783DF91CF911F910F91FF90EF9088
:107770000895CF93DF93CDB7DEB7EE97CDBFDEBFD1
:1077800088ED90E084BF9093610080E094E2A4EFE4
:10779000B0E08093112890931228A0931328B093FF
:1077A000142880910206866080930206809100066C
:1077B000816080930006809102068F7C8093020690
:1077C0008091A0008F788093A00080910206806154
:1077D000809302061092E20581E08093E40583E045
:1077E0008093010A8FEF90E08093260A9093270AF6
:1077F00080E890E08093380A9093390A80933A0A9F
:1078000090933B0A80933C0A90933D0A8BE08093CF
:10781000000A8091E50581608093E5058091E5058A
:1078200082608093E505E0E8FAE037E02FEF90E82A
:1078300085E031832487958780837096E03C0AE059
:10784000F007B9F780E094E08093DE2A9093DF2A76
:107850008091DE2A9091DF2A2FEF30E0B9010E945B
:10786000B1506093DC2A7093DD2A8091DE2A9091DA
:10787000DF2AE8EEF3E0BF010E94B1506093D42A02
:107880007093D52A8091DE2A9091DF2ABF010E9451
:10789000B1508093D22A9093D32A2093BC0A30937C
:1078A000BD0A8091B50A81608093B50A84E0809317
:1078B000B00A8091B00A81608093B00A78941092E7
:1078C000092E40E050E0BA0184EC9DE20E94D128EC
:1078D00088E280930B2E8093082E85E38093072EF9
:1078E00084E380930A2E87E890E080930C2E909397
:1078F0000D2E80EF90E080930E2E90930F2EE8EEE9
:10790000F7E09490E9EEF7E09A941FEF911609F4EE
:107910007EC014915F0122E0A20EB11C31968490CA
:10792000082D0F7784EC9DE20E94CB0F8091FB2DF8
:1079300087FD09C0E091DF2DF091E02D80819091CD
:10794000F62D89238083E091E12DF091E22D808155
:107950009091F82D89238083612F84EC9DE20E9411
:10796000190FE091E12DF091E22D80819091F72D9A
:10797000892B8083F501D12CC12C10E0C016D106D3
:10798000FCF48091F92D7F01823089F48091F42DEF
:10799000882369F0DF016D917D917D0184EC9DE28A
:1079A0000E94D40EEFEFCE1ADE0AF701E7CFBFEF49
:1079B000EB1AFB0A649184EC9DE20E94190FF2CF4E
:1079C0008091FB2D87FD09C0E091DF2DF091E02D26
:1079D00080819091F52D892B808384EC9DE20E941B
:1079E000BA0FF501E00FF11F87FE8ECF7F010FEF79
:1079F000E01AF00A649170E06F3F710511F464EFD2
:107A000071E090E080E00E942D07F7017DCF60E0FB
:107A100084EC9DE20E946B1070E060E084EC9DE2DB
:107A20000E947C1882E08093D82D8093D92D8CE021
:107A30000E943D2B91E0811101C090E090931528A8
:107A400063E0811101C061E084EC9DE20E946B1053
:107A500081E00E94402B62E070E08FE00E948F0581
:107A600062E070E084E00E948F0562E070E085E0F3
:107A70000E948F058CE090E00E94F8558C0145E053
:107A800064E00E94761E0093602A1093612A62E0EF
:107A900070E086E00E948F0582E190E00E94F85538
:107AA000FC011282138214821582BAE0AB2EB12C33
:107AB000A682B782108614EEC12E1EEED12EC08291
:107AC000D18280935C2A90935D2A86E0818BCF01DE
:107AD0000E949A09E0915C2AF0915D2A02E3E02E6F
:107AE000F12CE682F78262E070E087E00E948F0569
:107AF00062E070E08CE00E948F058CE090E00E94D4
:107B0000F8558C014CE067E00E94761E0093562ADF
:107B10001093572A62E070E08EE00E948F0582E1A8
:107B200090E00E94F855FC011282138214821582A3
:107B3000A682B7821086C082D18280935A2A9093FF
:107B40005B2A8EE0818BCF010E949A09E0915A2A2C
:107B5000F0915B2AE682F7828091C22D9091C32D2D
:107B60000E94945686E090E00E94F8558C0180E2D5
:107B7000D8018C9384E69CE211968D939C93129786
:107B800013961C92139780E290E014968D939C9329
:107B900015970093C22D1093C32D84E69CE20E949A
:107BA000B70D99249394F8019382C8010E94EE0DB9
:107BB00061E086E00E94EB1E61E085E00E94EB1E22
:107BC00061E084E00E94EB1E61E087E00E94EB1E12
:107BD00062E082E00E94EB1E62E080E00E94EB1E09
:107BE00061E083E00E94EB1E61E081E00E94EB1EF9
:107BF00082E190E00E94F855FC0112821382148207
:107C00001582A682B7821086C082D18280934F2AC5
:107C10009093502A8FE0818BCF010E949A09E091C6
:107C20004F2AF091502AE682F78260914B2869250D
:107C300084E00E941D1F60E087E00E941D1F61E03C
:107C400083E00E941D1F61E081E00E941D1F60E033
:107C500086E00E941D1F60E085E00E941D1F1092BB
:107C60009E2A61E070E080E10E948F0570E060E094
:107C700080E10E94F20561E070E081E10E948F05E1
:107C800070E060E081E10E94F20562E070E082E075
:107C90000E948F0561E270E382E00E94310462E09D
:107CA00070E083E00E948F0580EA9AE08093442C84
:107CB0009093452C8091A00A8E7F8093A00A909289
:107CC000A60A1092A10A84E08093A00A80E090E0C6
:107CD000A4E0B0E08093582C9093592CA0935A2C98
:107CE000B0935B2C8091A00A8E7F8093A00A809134
:107CF000A00A8670F0E48F2EF2E49F2EFFE0AF2EF4
:107D0000B12C853070F490E0FC01EE0FFF1FE80FFE
:107D1000F91FE950F14180819181A2814C01AA2E85
:107D2000B12C950144275527C501B401882799270F
:107D3000C12CD12C7601E394F1E0CF1AD108E108EF
:107D4000F108613071058105910539F4C501B4016F
:107D5000A70196010E942851EFCF2093462C309323
:107D6000472C4093482C5093492C60934A2C709395
:107D70004B2C80934C2C90934D2CC092522CD09233
:107D8000532CE092542CF092552C6115710581050D
:107D9000910561F0615071098109910960934A2C44
:107DA00070934B2C80934C2C90934D2C20934E2C05
:107DB00030934F2C4093502C5093512C232B242B39
:107DC000252B21F4C0904A2CD0904B2CC092AC0AA9
:107DD000D092AD0A1092AA0A1092AB0A8091A00A22
:107DE00081608093A00A87E69CE18093562C909353
:107DF000572C81E08093A60A8093A50A8091A00A5F
:107E00008E7F8093A00A8091A00A867090E9C92E87
:107E100090EDD92E93E0E92EF12C853060F490E0BE
:107E2000FC01EE0FFF1FE80FF91FE851F141C08080
:107E3000D180E280F12C80E090E0A1E0B0E080937E
:107E4000522C9093532CA093542CB093552C970103
:107E5000442755272093462C3093472C4093482C99
:107E60005093492CC701B6018827992760934A2C63
:107E700070934B2C80934C2C90934D2C21153105F5
:107E80004105510589F1412C512C32016394530174
:107E9000420101E0801A9108A108B1086130710522
:107EA0008105910549F4C701B601A50194010E941D
:107EB000285124013501EBCF4092522C5092532C83
:107EC0006092542C7092552C2093462C3093472C62
:107ED0004093482C5093492C60934A2C70934B2C20
:107EE00080934C2C90934D2C8091522C9091532C3C
:107EF000A091542CB091552C0197A109B109809300
:107F0000522C9093532CA093542CB093552C409109
:107F10004A2C50914B2C60914C2C70914D2C41155A
:107F200051056105710561F04150510961097109FF
:107F300040934A2C50934B2C60934C2C70934D2CB7
:107F40004091462C5091472C6091482C7091492CBF
:107F500040934E2C50934F2C6093502C7093512C87
:107F6000452B462B472B21F480914A2C90914B2C8A
:107F70008093AC0A9093AD0A1092AA0A1092AB0AB1
:107F80008091A00A81608093A00A87E79AE180939C
:107F9000AE2D9093AF2D1092B02D1092B12D8BEA93
:107FA00092E38093B82D9093B92D81E197E280936D
:107FB000B22D9093B32D0091432A1091442A8091C1
:107FC0009B2D90919C2DDC01ED91FC910684F78511
:107FD000E02D42E15AE760E070E0099510929D2D96
:107FE00010929E2D0093A72D1093A82D0E945D073F
:107FF0006093A82A7093A92A8093AA2A9093AB2A07
:10800000611571058105910511F00E948C508091D8
:10801000372881110E94D93181E00E946D2B2224E2
:108020002394312C0E945D076093FC2C7093FD2CEF
:108030008093FE2C9093FF2C8091452890914628A8
:108040008091C32A9091C42A2091C52A211109C088
:1080500021E0009709F020E02093C22A21E020933C
:10806000C52A2091C22A28171906C1F061E0892B80
:1080700009F460E087E00E941D1F61E08091C32A3F
:108080009091C42A892B09F460E06093C22A809100
:108090004B28882319F086E00E941D1F8091C12A79
:1080A000882309F48DC01092C12A809145289091AF
:1080B0004628892B29F08091D12A882309F46DC0A4
:1080C00020911628309117286091462A7091472AEE
:1080D0008091482A9091492A032E000C440B550B9D
:1080E0000E9428516093462A7093472A8093482A19
:1080F0009093492A8091F02C9091F12C019702974E
:1081000008F053C0E0914028F0914128CF010A9631
:1081100008E010E0B8010E94A6559C01220F331F11
:108120002159354DCF010996B8010E94A655FC0191
:10813000EE0FFF1FE159F54DD9018D919C912081E2
:108140003181821B930B865A9F4F80931628909300
:1081500017288091E42A8823C1F08091452A22EED5
:108160003FEF811102C02EE130E0809116289091FE
:108170001728820F931F80931628909317288091B9
:10818000452A91E089278093452A8091A02A882357
:1081900079F01092A02A0E94652780E090E0892B58
:1081A00009F440CF0E9400003ACF90E080E0CBCFAE
:1081B00080914B28882389F381E08093A12AEDCF19
:1081C0008091C02A882319F00E940228E6CF80916E
:1081D000BF2A882381F10E9402286091382870917B
:1081E000392880913A2890913B280E943F540E9460
:1081F0003D526B017C011C141D041E041F046CF60F
:108200008091BD2A9091BE2A8C33910554F08C192F
:108210009D0997FF03C091958195910903970CF4EF
:10822000BCCF40E0C701B6010E94C221C092BD2A66
:10823000D092BE2AB2CF8091B52A81110DC00E9482
:108240005D076093B12A7093B22A8093B32A90930A
:10825000B42A81E08093B52A4091B12A5091B22A84
:108260006091B32A7091B42A4115510561057105D9
:10827000E1F08091FC2C9091FD2CA091FE2CB0910E
:10828000FF2C841B950BA60BB70B813D9740A105D6
:10829000B10558F080E00E943D231092B12A10925F
:1082A000B22A1092B32A1092B42A80919B2D9091F9
:1082B0009C2DDC01ED91FC910084F185E02D099568
:1082C000181619060CF010C180919B2D90919C2DD1
:1082D000DC01ED91FC910284F385E02D0995182FC6
:1082E00087FD2FC080919D2D90919E2D892B49F562
:1082F0008091AC2D9091AD2D892B19F52091A42D55
:1083000080E8820F8037E8F4822F8F7090E001962A
:108310008093A92D9093AA2D4091A72D5091A82D1F
:1083200031E04115510521F08417950709F030E03F
:108330003093AB2D207F2093A32D20929D2D309242
:108340009E2D80919D2D90919E2D8130910509F457
:1083500065C08230910509F488C0892B79F5912F89
:10836000103F08F4907F9093A32D80E8890F803709
:1083700050F41093A42D212F2F702F5F30E0209305
:10838000A92D3093AA2D2091A72D3091A82D81E001
:108390002115310541F04091A92D5091AA2D421788
:1083A000530709F080E08093AB2D903E69F148F4CB
:1083B000903931F1903B41F1903859F11093A22D51
:1083C00074CF983F29F0D0F386E0890F8330B0F75F
:1083D000E091B82DF091B92D309781F321E09B3FCA
:1083E00009F020E041E09C3F09F040E061E09A3F65
:1083F00009F060E081E0983F09F080E00995DECF68
:1084000020929F2D3092A02D20929D2D30929E2D56
:10841000D5CF10929F2D1092A02DF6CF8091A32D35
:10842000803919F068F4803879F417FD0DC0E2E066
:10843000F0E0E0939D2DF0939E2D1093A12DBECFE3
:10844000803B39F0803E89F310929D2D10929E2D35
:10845000B5CF17FDF9CF1093A12DE2E08E2E912C10
:1084600080929D2D90929E2DA9CF8091A32D803931
:1084700019F0E8F4803841F717FDE6CF8091AB2D75
:1084800020919F2D3091A02D232B11F011111CC094
:10849000E091B02DF091B12D8823B1F23097A1F287
:1084A000412F6091A12D8091A92D0995CDCF803BC1
:1084B00091F0803E49F68091AB2D882329F2E0911E
:1084C000B42DF091B52DEACFE091AE2DF091AF2D06
:1084D0008111E4CFB9CF8091AB2DE091B22DF09115
:1084E000B32D8111DBCFB0CF00914F2A1091502ACC
:1084F000D80118968C9180FD13C00E945D07F80189
:10850000C184D284E384F4846C197D098E099F09A7
:1085100060934B2A70934C2A80934D2A90934E2A55
:10852000C0904B2AD0904C2AE0904D2AF0904E2AD1
:10853000C8010E94310980914A2A811116C1809197
:108540004F2A9091502A0E942909811107C0F8EC06
:10855000CF16D104E104F1040CF407C1809137284F
:10856000882309F4F3C00E945D076093A82A7093E2
:10857000A92A8093AA2A9093AB2A8091A72A8823BC
:1085800009F4E4C080E00E946D2B8091AF2A9091A5
:10859000B02A01968093AF2A9093B02A6BE070E0E6
:1085A0000E94A655892B99F483E00E9435069C0110
:1085B00091E02115310509F090E080911828981775
:1085C00031F090931828232B11F40E94B127809149
:1085D000AF2A9091B02A67E070E00E94A655892BDF
:1085E000D1F58091602A9091612A0E94621E6B01F0
:1085F0008090F02C9090F12C12E0811A91086090FC
:10860000DD2C7090DE2C22E0621A710800915E2A47
:1086100010915F2A0617170709F481C1CB018170F9
:108620009927892B09F07BC180913728882309F489
:1086300009C10E945D076093A82A7093A92A8093BC
:10864000AA2A9093AB2A8091A72A882309F4FAC01A
:1086500080E00E946D2B8091452890914628892BBF
:1086600009F099C38091AF2A9091B02A6DE070E033
:108670000E94A6558C01892B09F08DC38091672A31
:10868000811105C00E945D0781E08093672A85E122
:108690000E94DC069C01265031092FA738AB60E010
:1086A00074E0681B790B072E000C880B990B263F92
:1086B000334008F44FC30E9475526B017C01C09295
:1086C000C22CD092C32CE092C42CF092C52CC09244
:1086D000632AD092642AE092652AF092662A8091F9
:1086E000622A882309F414C584E1E2E8FEEEDE0183
:1086F000559601900D928A95E1F784E1E6E9FEEE48
:10870000DE01119601900D928A95E1F720E030E0AC
:1087100040EA50E4C701B6010E94C65187FDEEC48D
:1087200020E030E44EE754E4C701B6010E947D53D7
:108730004E0159E1850E911C18160CF0E3C3A8E810
:108740008A2EA3E19A2EA12CB12CDDC481E0809366
:108750004A2A80914B288823F9F008ECC016D104EE
:10876000E104F104CCF40E94B12780914A2A8823C5
:1087700009F40BCFE0914F2AF091502A808580FFB9
:1087800004CF10924A2A10924B2A10924C2A10922F
:108790004D2A10924E2AF9CE11E060E081270E9406
:1087A000072B80914B28882309F442C01092C32ADA
:1087B0001092C42A60E087E00E941D1F8091452826
:1087C00090914628892B59F5E091442CF091452C45
:1087D00080818E7F8083168380818E7F8083168345
:1087E0008091462C9091472CA091482CB091492C17
:1087F00080934E2C90934F2CA093502CB093512CDF
:10880000892B8A2B8B2B79F08091522C9091532CB1
:10881000848795871286138680818160808381E0BA
:108820008093A02AA2CF80914A2C90914B2CF0CF1C
:10883000209145283091462881E02130310581F38F
:1088400080E0EECFC601801B910B21E030E01816CE
:10885000190614F02FEF3FEF42E08416910408F060
:10886000CDC08091832A9091842A08964091812AD4
:108870005091822A841B950B68E070E00E94A655F7
:10888000AC01DC01AA0FBB1FFD01E159F54D0081D0
:108890001181F80117FF07C0EE27FF27E01BF10B3E
:1088A0003195219531092130310549F4E531F10542
:1088B0004CF4E830F10544F52E0F3F1F0FC0E631B0
:1088C000F105FCF0C901880F991F280F391F2E0FE1
:1088D0003F1F2F31310514F02EE130E017FF03C0A8
:1088E000319521953109A159B54D2D933C93809136
:1088F0004B28882361F0BA0181E090E00E9469076B
:108900000AC0E930F105C4F2220F331FD5CF61E070
:1089100080E00E94A322C0925E2AD0925F2A8091BA
:108920005C2A90915D2A0E94310980915A2A909187
:108930005B2A0E94310980915C2A90915D2A0E94F5
:108940002909182F80915A2A90915B2A0E9429099F
:10895000B82E1123C9F080913728882371F00E9426
:108960005D076093A82A7093A92A8093AA2A9093FE
:10897000AB2A8091A72A81116BCE8091592A882336
:1089800009F499C01092592A8091562A9091572A39
:108990000E94621E6B010091542A1091552A0617FD
:1089A000170709F4F9C0CB0181709927892B09F0C9
:1089B000F3C080913728882371F00E945D0760938F
:1089C000A82A7093A92A8093AA2A9093AB2A80910F
:1089D000A72A81113DCEC601801B910B18161906DE
:1089E0000CF0AEC081E090E02091832A3091842A7F
:1089F000820F931F97FFA7C00896FCCF52E0651621
:108A0000710408F043C08091832A9091842A0896CB
:108A10004091812A5091822A841B950B68E070E076
:108A20000E94A655AC01FC01EE0FFF1FDF01AF5DF8
:108A3000B74D8D919C91280F391F29833A832D8A38
:108A40003E8ADE0122303105D4F0119688E090E0B4
:108A500089A79AA78D919C911197089714F0DE0130
:108A60009996EF5DF74D8D919C91808391838091D4
:108A70004B28882331F0BA0182E090E03FCF559631
:108A8000E5CF61E080E00E94252245CF8091E72A72
:108A90009091E82A820F931F97FF02C00A96FCCF9D
:108AA0006AE070E00E94A6558093E72A9093E82A36
:108AB0000E94042130CF82E088169104E0F4809176
:108AC000832A9091842A08962091812A3091822AC3
:108AD000821B930B68E070E00E94A655FC01EE0F2C
:108AE000FF1FE159F54D10821182AC0160E080E07A
:108AF0000E94A32249CF92E069167104E0F48091AC
:108B0000832A9091842A08962091812A3091822A82
:108B1000821B930B68E070E00E94A655FC01EE0FEB
:108B2000FF1FEF5DF74D20823182AC0160E080E0F5
:108B30000E94252229CF1092582A0E94582624CF1D
:108B40008FEF9FEF51CF877099278093832A90935F
:108B5000842AA2E08A16910408F08CC0089620911D
:108B6000812A3091822A821B930B68E070E00E9478
:108B7000A65520914B28222331F0BC0181E090E0E2
:108B80000E94690705C0AC0161E080E00E94A32259
:108B9000C092542AD092552AE2E08E16910408F42D
:108BA0004CC0F2E06F16710408F447C0809145286C
:108BB00090914628019709F440C08091532A811171
:108BC0003CC000915A2A10915B2AD80118968C91CA
:108BD00080FD33C00E945D07F80101851285238561
:108BE0003485601B710B820B930B653F71408105CF
:108BF000910518F181E08093532A8091512A909138
:108C0000522A0196833091050CF06BC08093512A53
:108C10009093522AE091512AF091522AEE0FFF1FB1
:108C2000EE0FFF1FEA5FF0416081718182819381C5
:108C30000E943D52CB010E947324BB2009F40BCD4E
:108C400080913728882371F00E945D076093A82ADD
:108C50007093A92A8093AA2A9093AB2A8091A72A7D
:108C60008111F6CC8091532A882309F43FC01092D9
:108C7000532AF1CCB2E06B167104C8F40896209127
:108C8000812A3091822A821B930B68E070E00E9457
:108C9000A65520914B28222321F0BC0182E090E0D0
:108CA0006FCFAC0161E080E00E94252271CF49E1E5
:108CB00050E063E070E084E890E00E94A11A8091A7
:108CC000832A9091842A01960E94B81F8FEF9FEF0C
:108CD0008093D62D9093D72D8093D42D9093D52D1E
:108CE00057CF1092512A1092522A94CF02E0801648
:108CF000910408F4B0CC12E06116710408F4ABCC16
:108D00008091832A9091842A019689839A832D8A5F
:108D10003E8AFE010297E4F0319688E090E089A750
:108D20009AA780819181089714F0FE01B9968081FD
:108D3000918120913E2830913F288217930709F4B2
:108D40008ACC80933E2890933F280E94BA2083CCFF
:108D50007596E3CF0E947552AB01BC018EEB9CE28D
:108D60000E94C71C6B017C012091632A3091642A08
:108D70004091652A5091662A0E9459510E943D52A5
:108D80009B0177FF04C022273327261B370B233094
:108D900031050CF09CCC8091AF2A9091B02A6BEBFE
:108DA00070E00E94A655892B11F40E946E2F20912D
:108DB000AF2A3091B02AC90165E270E00E94A65541
:108DC000892B09F085C349EE5CE266ED7CE282E026
:108DD00090E00E94A407182F8823B1F18091DD2C28
:108DE0009091DE2C0297029778F58091DC2C8823F5
:108DF00001F12092212830922228209223283092BB
:108E00002428209225283092262820922728309244
:108E100028282092292830922A2820922B28309224
:108E20002C2820922D2830922E2820922F28309204
:108E3000302880914B28882309F497C26FEF7FEF89
:108E400082E090E00E94690746ED5CE269EE7CE218
:108E500090E080E00E94A407882309F4ADC68091C9
:108E6000F02C9091F12C0297029778F58091EF2CDD
:108E7000882301F110926F2A1092702A1092712AA1
:108E80001092722A1092732A1092742A1092752AE4
:108E90001092762A1092772A1092782A1092792AC4
:108EA00010927A2A10927B2A10927C2A10927D2AA4
:108EB00010927E2A80914B28882309F45DC26FEFBF
:108EC0007FEF81E090E00E94690780913728882336
:108ED00009F459C20E945D076093A82A7093A92AD9
:108EE0008093AA2A9093AB2A8091A72A882309F419
:108EF0004AC280E00E946D2B50C9850104301105E3
:108F000009F490C058018FEFA81AB80AD4012D9126
:108F10003D914D915D914D012BAB3CAB4DAB5EABAB
:108F2000CA01B9010E9475529B01AC01C701B6018B
:108F30000E94C65187FFE1CFAA0CBB1CAA0CBB1C28
:108F4000E1E0F0E0EC0FFD1FEA0DFB1D40805180D9
:108F5000628073805801AA0CBB1CAA0CBB1CE1E008
:108F6000F0E0EC0FFD1FAE0EBF1ED5016D917D919F
:108F70008D919C910E9475520E943D526BA77CA7D7
:108F80008DA79EA7D50154960D911D912D913C91D1
:108F900057970BAF1CAF2DAF3EAFC301B2010E947C
:108FA00075520E943D524B015C010BA51CA52DA5DD
:108FB0003EA5801A910AA20AB30A8FAA98AEA9AE5A
:108FC000BAAEC701B6010E943D528BAC9CACADACB1
:108FD000BEAC681979098A099B092FA938AD49AD3A
:108FE0005AAD0E948A552BA93CA94DA95EA9281902
:108FF00039094A095B090E94C5508BA49CA4ADA401
:10900000BEA4820E931EA41EB51E8BA69CA6ADA662
:10901000BEA6481459046A047B0424F44BA65CA63B
:109020006DA67EA66BA57CA58DA59EA50E947552FA
:10903000AFA4B8A806EFA01603E0B00608F4AFC0CE
:109040006093B62C7093B72C8093B82C9093B92C66
:109050000E943D5220914728309148282617370713
:1090600009F46BC16093472870934828809349287E
:1090700090934A280E9475526FA778AB89AB9AAB40
:109080008090312890903228A0903328B0903428D6
:109090008BAA9CAAADAABEAA9B01AC0160EC71EEA2
:1090A00084E69CE40E94CB51A50194010E94825366
:1090B00020E030E044EB52E40E94CB510E943F5448
:1090C0000E9444526B017C010091442C1091452C6C
:1090D000D8018C918E7F8C938C918670823009F4AC
:1090E000ABC0843009F464C0811169C054E0CC0C79
:1090F000DD1CEE1CFF1C5A95D1F761C0BEE18B2E22
:10910000912CA12CB12C8BA69CA6ADA6BEA68ACF75
:10911000C701B6010E943D529B01AC0125503109A7
:1091200041095109A4E5B1E00E94E45027EF33E082
:1091300040E050E00E94C550CA01B901675E7F4F10
:109140008F4F9F4F0E9475526B017C0120E030E0F1
:1091500040EF51E40E947D5318169CF420E030E06B
:1091600044EB53E4C701B6010E94C65187FF10C00B
:10917000C701B6010E943D526BA77CA78DA79EA791
:1091800051CFC12CD12CF0EFEF2EF1E4FF2EF0CF18
:10919000C12CD12CE4EBEE2EE3E4FE2EE9CFAB01A3
:1091A000BC0182EB9CE20E94C71C0E94B05250CFCF
:1091B00072E0F694E794D794C7947A95D1F7812C0E
:1091C000912C5401A3948092522C9092532CA092F3
:1091D000542CB092552C9701442755272093462CA8
:1091E0003093472C4093482C5093492CC701B6012B
:1091F0008827992760934A2C70934B2C80934C2C92
:1092000090934D2C2115310541055105A9F12401FB
:109210003501A1E04A1A51086108710861307105F1
:109220008105910589F4C701B601A30192010E944D
:10923000285153014201EBCF63E0CC0CDD1CEE1C46
:10924000FF1C6A95D1F7BBCF8092522C9092532C81
:10925000A092542CB092552C2093462C3093472C3E
:109260004093482C5093492C60934A2C70934B2C7C
:1092700080934C2C90934D2C8091522C9091532C98
:10928000A091542CB091552C0197A109B10980935C
:10929000522C9093532CA093542CB093552C409166
:1092A0004A2C50914B2C60914C2C70914D2C4115B7
:1092B00051056105710561F041505109610971095C
:1092C00040934A2C50934B2C60934C2C70934D2C14
:1092D0004091462C5091472C6091482C7091492C1C
:1092E00040934E2C50934F2C6093502C7093512CE4
:1092F000452B462B472B21F480914A2C90914B2CE7
:10930000F801848795871286138680818160808327
:109310008091452890914628892B79F42BA93CA966
:109320004DA95EA96FA578A989A99AA90E94CB51D8
:109330000E943D5240E00E94C2218091372888233C
:1093400009F429CD0E945D076093A82A7093A92A89
:109350008093AA2A9093AB2A8091A72A882309F4A4
:109360001ACD80E00E946D2B16CD50E040E061E008
:1093700081E00E94252268CD50E040E061E081E07C
:109380000E94A322A2CD61E08091DD2C9091DE2C81
:10939000019709F460E083E00E941D1F61E0809165
:1093A000F02C9091F12C019709F460E081E00E948B
:1093B0001D1F8091DD2C9091DE2C0297029738F0D2
:1093C0008091F02C9091F12C0297029750F58091AA
:1093D000832A9091842A8093812A9093822A809173
:1093E000DD2C9091DE2C0297029740F486ED9CE2F2
:1093F0000E94361A682F83E00E941D1F8091F02C76
:109400009091F12C0297029710F00C94CD4089EEC8
:109410009CE20E94361A682F81E00E941D1F0C9466
:10942000CD4080914B28882309F446C080915C2868
:1094300090915D28A0915E28B0915F28892B8A2B9E
:109440008B2B51F40E945D0760935C2870935D281C
:1094500080935E2890935F2881E0809362288091BA
:10946000DD2C9091DE2C0297029770F08091DF2C1A
:109470009091E02C0297029738F480914B28882332
:1094800009F181E08093802A8091F02C9091F12C59
:109490000297029708F4A3CF8091F22C9091F32CBD
:1094A0000297029708F09BCF80914B28882369F0A0
:1094B00081E080937F2A93CF81E00E943D230E9428
:1094C0000421CDCF0E94E52ADFCF0E94F62A87CF64
:1094D000C90165E370E00E94A655892BC9F480910B
:1094E0005C2890915D28A0915E28B0915F28892B1F
:1094F0008A2B8B2B69F00E945D0720915C283091AC
:109500005D28621B730B6D32714014F00E94D023F2
:109510008091AE2A811135C11FA68091AF2A90910A
:10952000B02A60E177E20E94A655892BA9F48091C8
:109530004B28882309F4B4C18091FC2C9091FD2C18
:10954000A091FE2CB091FF2C8093A82A9093A92A79
:10955000A093AA2AB093AB2A8091A72A882309F462
:10956000E3C08091A32A9091A42AA091A52AB0914A
:10957000A62A4091FC2C5091FD2C6091FE2C7091FC
:10958000FF2C481B590B6A0B7B0B4F3151056105B2
:10959000710508F4C9C04E96A11DB11D8093A32A80
:1095A0009093A42AA093A52AB093A62A8091372845
:1095B000882309F4B9C06091952A7091962A072EE4
:1095C000000C880B990B0E9475526B017C01609115
:1095D000CE2D7091CF2D072E000C880B990B0E9479
:1095E00075529B01AC01C701B6010E94CB512B0102
:1095F0003C0120911D2830911E2840911F28509138
:1096000020280E94EF534B015C010091932A109196
:10961000942AC0908F2AD090902AE0901B28F09036
:109620001C2860918D2A70918E2A6C197D09072E55
:10963000000C880B990B0E947552A30192010E94A5
:1096400082532B013C01B601DD0C880B990B0E9463
:1096500075529B01AC01C301B2010E945A510E9494
:109660003D522B016091912A7091922A601B710BDF
:10967000072E000C880B990B0E947552A5019401CE
:109680000E9482534B015C01B801110F880B990BAA
:109690000E9475529B01AC01C501B4010E945A5150
:1096A0000E943D5240918B2A50918C2AE091892A48
:1096B000F0918A2A82019B01BF0184EC9DE20E9405
:1096C00004188091192890911A282091952A309198
:1096D000962A280F391F2093952A3093962A409175
:1096E000CE2D5091CF2D840F951F82179307E4F450
:1096F0008091872A9091882A01962091852A30911D
:10970000862A2F5F3F4F2093852A3093862A64E074
:1097100070E00E94A6558093872A9093882A8091B2
:10972000372881110E94D9318091AE2A10E000E0E3
:10973000882309F4E4C0E091AC2AF091AD2A628557
:1097400087E00E941D1F8091AC2A9091AD2ADC0118
:109750001A962C91222319F08FA48110C8C090E092
:1097600080E00E94BA208091A22A811104C090E07A
:1097700080E00E94C21F81E08093A22A0FEF1FEFBA
:10978000BEC00091AC2A1091AD2A0E945D072B014A
:109790003C01D80114968C9130E020E08B3218F413
:1097A0000E9435069C0191E02130310509F490E0DA
:1097B000F801928786810E94DC062FEF33E0281B98
:1097C000390BD80118962D933C9319971A968C90C3
:1097D0001A978FA6811015C01F961D921D921D927B
:1097E0001C9252978FEF9FEF53968D939C935497B3
:1097F0001D968D939C931E9718961D921C921997F7
:109800008CCEF80187859089A189B289892B8A2B12
:109810008B2B21F44786508A618A728AF801E3848F
:10982000F484E586F686C8010E942624D8011B969A
:109830008D939C931C971F964D915D916D917C919A
:109840005297411551056105710509F465CE441A19
:10985000550A660A770A55962D913C915697032E24
:10986000000C440B550B241535054605570508F02B
:1098700053CE53962D913C918217930709F44CCE09
:10988000E816F90609F048CEF8011786108A118A01
:10989000128AE38AF48A8FEF9FEF858796873DCE01
:1098A00080913728882309F457CE8091A72A811107
:1098B00058CE0E945D070091A82A1091A92A2091F4
:1098C000AA2A3091AB2A601B710B820B930B613E6D
:1098D00073498440910508F427CF81E08093A72A3B
:1098E00070E060E084EC9DE20E947C1835CE0E941E
:1098F00026248C0181E08093A12A1092A22A8091D3
:10990000A02A882321F01092A12A0C94CD408091A6
:10991000BF2A81110C94CD4080914B2881110AC03F
:109920008091AE2A811106C080919F2A882311F46C
:109930000C94CD408091A12A8823E9F080919E2A41
:10994000882331F060E085E00E941D1F10929E2A5E
:109950001092A12A81E080939D2A80919F2A8823DA
:1099600009F45BC060E080913528909136280E9410
:1099700061200E94D02360914728709148288091EF
:10998000492890914A2822E030E040E050E00E94CF
:10999000C550CA01B9010E947552209131283091F9
:1099A000322840913328509134280E94CB5120E036
:1099B00030E44CE955E40E947D5308EC10E087FF49
:1099C00002C008E512E080919D2A882311F40C94CE
:1099D000CD400E94FE06AB01BC01C801110FAA0BCD
:1099E000BB0B0091992A10919A2A20919B2A3091C1
:1099F0009C2A800F911FA21FB31F481759076A079F
:109A00007B0710F40C94CD4010929D2A70E060E02A
:109A100080E10E94F2050C94CD40D090AE2ADD206A
:109A200019F060E0C801A3CFE0903E28F0903F28F5
:109A30008091972A9091982A01978093972A9093E2
:109A4000982A0091402810914128181619060CF404
:109A500055C080913C2890913D288330910509F4B0
:109A600079C0A8F4009140281091412881309105D7
:109A7000F1F0029769F100914028109141280F5FA1
:109A80001F4F0E151F05ACF110E000E032C084300E
:109A9000910509F475C0059771F70E94E14F892F70
:109AA000990F990BB7010E94A6558C0127C0015050
:109AB0001109C701019717FD03C00E151F050CF012
:109AC0008C01DD24D39480179107C1F0D12C16C0EE
:109AD00080914228882391F10F5F1F4F17FF31C0FB
:109AE00081E08093422810E000E0D0904228DD2001
:109AF00029F0DD24D3940115110541F76D2DC8011E
:109B00000E9461208091972A9091982A1816190630
:109B10000CF42FCF8091DD2C9091DE2C01970297D1
:109B200008F047C0000F111FF801EF5DF74D80816D
:109B300091818093972A9093982A1BCF0150110905
:109B4000CDCF0E151F058CF287010150110910921F
:109B50004228CBCF01E0E016F10409F495CF8091C3
:109B60004028909141288C010E5F1F4F0E151F0554
:109B70000CF4BFCF8C010095109501701127B9CF5F
:109B800080914328909144280196B7010E94A655E0
:109B90008093432890934428FC01EE0FFF1FE45B61
:109BA000F74D00811181DD24D394892B09F4A6CFD0
:109BB0008DCF81E090E0BDCF111187C910CCCF933C
:109BC000DF93DC012D91FB013191EC013883EB0136
:109BD000288341505109CD01BF01141615068CF39D
:109BE000DF91CF910895B0E0A0E0E9EFFDE40C949F
:109BF00001516C01D62FC72F8A017901F90109950E
:109C0000B80197FF15C08D2F9C2FF701099597FD7F
:109C100008C0B801C601F701099597FD16C0DC2DF3
:109C2000CD2D8D2F9C2FCDB7DEB7E8E00C941A51C7
:109C30008D2F9C2FF70109951816190694F3B8017A
:109C4000C601F701099597FDEACFD02FC12FE9CFC3
:109C5000A8E0B0E0EEE2FEE40C94F7508C014F83F4
:109C6000588759019A013195219531092D833E83F9
:109C70006F807884600E711E6730710578F58F8172
:109C80009885689F6001699FD00C789FD00C112443
:109C9000C00ED11E6C147D0420F02896E2E10C94D5
:109CA0001051730113C047012F813885821A930A1E
:109CB000B701C401F50109951816190654F44F812E
:109CC0005885B401C7010E94DF4D74010E151F05B0
:109CD00050F3EF81F8856E0E7F1EDCCFCB01969599
:109CE00087952F813885829F6001839FD00C929F3A
:109CF000D00C1124C00ED11ECB010197829F100100
:109D0000839F300C929F300C11247801E20CF31CDD
:109D10006730710509F442C0C70128016932710535
:109D2000B0F183E0769567958A95E1F7629F4001EF
:109D3000639F900C729F900C1124C401880F991F8F
:109D400089839A83AC01400F511FB801680D791DBA
:109D50009501C8010E94F34D2C01A601480D591D23
:109D60009194819491089501B601C601880D991DC1
:109D70000E94F34D6C01B701680D791D9501A70193
:109D8000C701E981FA818E1B9F0B0E94F34D95015B
:109D9000AC01B601C2010E94F34D6C014F815885A0
:109DA000B601C8010E94DF4D4301630127011982FA
:109DB0001A82EC14FD0408F446C0B801C601F5018E
:109DC00009951816190654F1892B71F44F8158859D
:109DD000B601C3010E94DF4D2F813885620E731ECC
:109DE00081E090E089839A83EF81F885CE0EDF1EB3
:109DF000E0CF892B71F44F815885B201C7010E94D1
:109E0000DF4D2D813E81420E531E81E090E089831B
:109E10009A83EB80FC80EC14FD04A8F0B801C70124
:109E2000F50109952D813E812E0D3F1D2B833C832D
:109E300097FFDFCF4F815885B701C6010E94DF4DE4
:109E4000EB80FC80CDCFEF81F8852E0E3F1E200EDB
:109E5000311E29813A81232B09F58214930408F0DD
:109E60001CCF740113C06701EF81F885CE1ADF0A99
:109E7000B701C601F50109951816190654F44F816A
:109E80005885B601C7010E94DF4D76010E151F05EA
:109E900050F38F819885880E991EDFCF4601861872
:109EA0009708A301401B510B841695060CF4A401DE
:109EB0001416150634F4B601641B750BC8010E9414
:109EC000DF4D92012E193F097901A101441955096D
:109ED0008F819885481B590B2417350708F4A90171
:109EE0001416150634F4B101641B750BC6010E94EB
:109EF000DF4DEF81F885E815F90548F4C401BF018D
:109F00000E94B1509501AF01C8010E94284E2F81D7
:109F100038852E153F0508F0C0CE81010E191F09A6
:109F2000C701B9010E94B150A3CE8F929F92AF9208
:109F3000BF92CF92DF92EF92FF92CF93DF93EC012B
:109F4000688179818A819B816115710581059105FF
:109F500021F464E279ED8BE597E02DE133EF41E008
:109F600050E00E94C55049015A019B01AC01A7EA8B
:109F7000B1E40E94E4506B017C01ACEEB4EFA501AA
:109F800094010E94F250DC01CB018C0D9D1DAE1D91
:109F9000BF1DB7FF03C00197A109B048888399830B
:109FA000AA83BB839F77DF91CF91FF90EF90DF90E3
:109FB000CF90BF90AF909F908F9008950E94954F43
:109FC000089587E698E20E94954F0895B0E0A0E0DA
:109FD0008093672890936828A0936928B0936A2893
:109FE00008958F929F92AF92BF92CF92DF92EF929D
:109FF000FF92CF93DF93EC01688179818A819B8105
:10A00000611571058105910521F464E279ED8BE517
:10A0100097E02DE133EF41E050E00E94C550490147
:10A020005A019B01AC01A7EAB1E40E94E4506B0124
:10A030007C01ACEEB4EFA50194010E94F250C60E73
:10A04000D71EE81EF91EF7FE06C081E0C81AD10827
:10A05000E10880E8F80AC882D982EA82FB82C70157
:10A06000B6019F77DF91CF91FF90EF90DF90CF9077
:10A07000BF90AF909F908F9008958F929F92AF92D4
:10A08000BF92CF92DF92EF92FF9260916B28709116
:10A090006C2880916D2890916E286115710581055D
:10A0A000910521F464E279ED8BE597E02DE133EF42
:10A0B00041E050E00E94C55049015A019B01AC01AA
:10A0C000A7EAB1E40E94E4506B017C01ACEEB4EF6E
:10A0D000A50194010E94F250C60ED71EE81EF91E7B
:10A0E000F7FE06C081E0C81AD108E10880E8F80A46
:10A0F000C0926B28D0926C28E0926D28F0926E2866
:10A10000C701B6019F77FF90EF90DF90CF90BF908F
:10A11000AF909F908F90089560936B2870936C28F8
:10A1200080936D2890936E28089503D0808199279D
:10A130000895FC01E050FC4E0895262FAF93BF9385
:10A14000E0E0F0E1328131FDFDCFDC01A050BC4EFA
:10A150002C932DE924BF23E020830196BF91AF917A
:10A160000895AA1BBB1B51E107C0AA1FBB1FA6175E
:10A17000B70710F0A61BB70B881F991F5A95A9F7B0
:10A1800080959095BC01CD010895052E97FB1EF496
:10A1900000940E94DC5057FD07D00E94285107FC14
:10A1A00003D04EF40C94DC50509540953095219599
:10A1B0003F4F4F4F5F4F08959095809570956195F3
:10A1C0007F4F8F4F9F4F08950E944A51A59F900D3A
:10A1D000B49F900DA49F800D911D11240895B7FF89
:10A1E0000C94E4500E94E450821B930B08952F922C
:10A1F0003F924F925F926F927F928F929F92AF9217
:10A20000BF92CF92DF92EF92FF920F931F93CF9363
:10A21000DF93CDB7DEB7CA1BDB0BCDBFDEBF099422
:10A220002A88398848885F846E847D848C849B84E6
:10A23000AA84B984C884DF80EE80FD800C811B81F4
:10A24000AA81B981CE0FD11DCDBFDEBFED0108952A
:10A25000A1E21A2EAA1BBB1BFD010DC0AA1FBB1F2A
:10A26000EE1FFF1FA217B307E407F50720F0A21B9C
:10A27000B30BE40BF50B661F771F881F991F1A9409
:10A2800069F760957095809590959B01AC01BD0133
:10A29000CF010895A29FB001B39FC001A39F700D8D
:10A2A000811D1124911DB29F700D811D1124911DDE
:10A2B00008955058BB27AA270E9471510C942B5324
:10A2C0000E941D5338F00E94245320F039F49F3F20
:10A2D00019F426F40C941A530EF4E095E7FB0C9451
:10A2E000EB52E92F0E943C5358F3BA1762077307E9
:10A2F0008407950720F079F4A6F50C9476530EF4B4
:10A30000E0950B2EBA2FA02D0B01B90190010C0185
:10A31000CA01A0011124FF27591B99F0593F50F49D
:10A32000503E68F11A16F040A22F232F342F4427F5
:10A33000585FF3CF469537952795A795F0405395ED
:10A34000C9F77EF41F16BA0B620B730B840BBAF0BD
:10A350009150A1F0FF0FBB1F661F771F881FC2F728
:10A360000EC0BA0F621F731F841F48F4879577953C
:10A370006795B795F7959E3F08F0B0CF9395880FF6
:10A3800008F09927EE0F9795879508950E94C75278
:10A3900008F481E008950E94DF510C942B530E9431
:10A3A000245358F00E941D5340F029F45F3F29F0D8
:10A3B0000C94EB5251110C9477530C941A530E9445
:10A3C0003C5368F39923B1F3552391F3951B550B37
:10A3D000BB27AA2762177307840738F09F5F5F4F78
:10A3E000220F331F441FAA1FA9F335D00E2E3AF0B7
:10A3F000E0E832D091505040E695001CCAF72BD0CF
:10A40000FE2F29D0660F771F881FBB1F261737071F
:10A410004807AB07B0E809F0BB0B802DBF01FF2751
:10A4200093585F4F3AF09E3F510578F00C94EB52F1
:10A430000C9477535F3FE4F3983ED4F38695779579
:10A440006795B795F7959F5FC9F7880F911D96950A
:10A45000879597F90895E1E0660F771F881FBB1F66
:10A46000621773078407BA0720F0621B730B840B13
:10A47000BA0BEE1F88F7E09508950E944452689445
:10A48000B1110C94775308950E94445388F09F575C
:10A4900098F0B92F9927B751B0F0E1F0660F771F08
:10A4A000881F991F1AF0BA95C9F714C0B13091F0FE
:10A4B0000E947653B1E008950C947653672F782F5D
:10A4C0008827B85F39F0B93FCCF3869577956795C3
:10A4D000B395D9F73EF490958095709561957F4F2F
:10A4E0008F4F9F4F0895E89409C097FB3EF49095D5
:10A4F0008095709561957F4F8F4F9F4F9923A9F05D
:10A50000F92F96E9BB279395F695879577956795EB
:10A51000B795F111F8CFFAF4BB0F11F460FF1BC02F
:10A520006F5F7F4F8F4F9F4F16C0882311F096E9C2
:10A5300011C0772321F09EE8872F762F05C0662370
:10A5400071F096E8862F70E060E02AF09A95660F29
:10A55000771F881FDAF7880F9695879597F90895E2
:10A560000E945E5390F09F3748F4911116F00C94BE
:10A57000775360E070E080E89FEB089526F41B16A7
:10A58000611D711D811D0C94F1520C940C53990F97
:10A590000008550FAA0BE0E8FEEF16161706E807AD
:10A5A000F907C0F012161306E407F50798F0621BCE
:10A5B000730B840B950B39F40A2661F0232B242BA3
:10A5C000252B21F408950A2609F4A140A6958FEFC2
:10A5D000811D811D089597F99F6780E870E060E014
:10A5E0000895882371F4772321F09850872B762FD4
:10A5F00007C0662311F499270DC09051862B70E097
:10A6000060E02AF09A95660F771F881FDAF7880FA7
:10A610009695879597F908959F3F31F0915020F4D2
:10A62000879577956795B795880F911D969587952E
:10A6300097F908959FEF80EC089500240A94161668
:10A64000170618060906089500240A941216130620
:10A65000140605060895092E0394000C11F48823AE
:10A6600052F0BB0F40F4BF2B11F460FF04C06F5FCA
:10A670007F4F8F4F9F4F089557FD9058440F551FA0
:10A6800059F05F3F71F04795880F97FB991F61F074
:10A690009F3F79F087950895121613061406551FEB
:10A6A000F2CF4695F1DF08C0161617061806991F57
:10A6B000F1CF869571056105089408950E94445371
:10A6C000A0F0BEE7B91788F4BB279F3860F41616D0
:10A6D000B11D672F782F8827985FF7CF86957795DC
:10A6E0006795B11D93959639C8F30895E894BB27F3
:10A6F00066277727CB0197F908950E94C75208F47F
:10A700008FEF08950E9495530C942B530E941D5374
:10A7100038F00E94245320F0952311F00C94EB5252
:10A720000C941A5311240C9477530E943C5370F3E9
:10A73000959FC1F3950F50E0551F629FF001729FE6
:10A74000BB27F00DB11D639FAA27F00DB11DAA1FF5
:10A75000649F6627B00DA11D661F829F2227B00D42
:10A76000A11D621F739FB00DA11D621F839FA00DCD
:10A77000611D221F749F3327A00D611D231F849F1D
:10A78000600D211D822F762F6A2F11249F57504074
:10A790009AF0F1F088234AF0EE0FFF1FBB1F661FEF
:10A7A000771F881F91505040A9F79E3F510580F0B8
:10A7B0000C94EB520C9477535F3FE4F3983ED4F340
:10A7C000869577956795B795F795E7959F5FC1F75C
:10A7D000FE2B880F911D9695879597F90895FA019C
:10A7E000EE0FFF1F309621053105A1F161157105AE
:10A7F00061F48038BFE39B0749F168949038810584
:10A8000061F08038BFEF9B0741F099234AF5FF3F85
:10A81000E1053105210519F1E8940894E795D9017E
:10A82000AA2329F4AB2FBE2FF85FD0F310C0FF5F2F
:10A8300070F4A695E0F7F73950F019F0FF3A38F4C4
:10A840009F779F930DD00F9007FC9058089546F086
:10A850000C941A5360E070E080E89FE308954FE79E
:10A860009F775F934F933F932F930E940E552F91A5
:10A870003F914F915F910E9482530C946B540E94C0
:10A880004453E8F09E37E8F09639B8F49E3848F41F
:10A89000672F782F8827985FF9CF869577956795EA
:10A8A00093959539D0F3B62FB1706B0F711D811D43
:10A8B00020F487957795679593950C94F1520C94B5
:10A8C0000C530C94775329F416F00C94EB520C941F
:10A8D00076530C941A530E944453A8F39638A0F769
:10A8E00007F80F92E8942BE33AEA48EB5FE70E94FF
:10A8F00098530F920F920F924DB75EB70F920E942E
:10A900005655E0EAF0E00E949D544F915F91EF911F
:10A91000FF91E595EE1FFF1F49F0FE57E0684427C1
:10A92000EE0F441FFA95E1F74195550B0E94D05464
:10A930000F9007FE0C94C4540895DF93CF931F9398
:10A940000F93FF92EF92DF927B018C01689406C017
:10A95000DA2EEF010E949553FE01E894A59125910E
:10A96000359145915591A6F3EF010E947151FE0179
:10A970009701A801DA9469F7DF90EF90FF900F91AB
:10A980001F91CF91DF9108959B01AC0160E070E0D1
:10A9900080E89FE30C94CB510C94EB520C940C5335
:10A9A0000E944453D8F39923C9F3940F511DA3F384
:10A9B0009150504094F059F0882332F0660F771F81
:10A9C000881F91505040C1F79E3F51052CF7880FCA
:10A9D000911D9695879597F908955F3FACF0983E45
:10A9E0009CF0BB27869577956795B79508F4B1607D
:10A9F0009395C1F7BB0F58F711F460FFE8CF6F5F75
:10AA00007F4F8F4F9F4FE3CF0C94775316F00C94EA
:10AA10000C530C941A5368940C94EB520E944453B8
:10AA2000A8F39923C1F3AEF3DF93CF931F930F9352
:10AA3000FF92C92FDD2788232AF02197660F771F01
:10AA4000881FDAF720E030E040E85FEB9FE38839C9
:10AA500020F0803E38F021968F770E945A51E8EC22
:10AA6000F0E004C00E945A51E5EFF0E00E949D54CE
:10AA70008B01BE01EC01FB2E6F5771097595771F95
:10AA8000880B990B0E94755228E132E741E35FE39E
:10AA90000E949553AF2D9801AE01FF900F911F9129
:10AAA000CF91DF910E9471510C942B53FA01DC017C
:10AAB000AA0FBB1F9B01AC01BF5728F422273327E5
:10AAC0004427507820C0B75190F4AB2F002446950E
:10AAD00037952795011CA395D2F3002071F0220F22
:10AAE000331F441FB395DAF30ED00C9459516130E3
:10AAF0007105A0E88A07B94630F49B01AC016627CE
:10AB0000772788279078309621F0208331834283FD
:10AB100053830895DB018F939F930E94E450BF916C
:10AB2000AF91A29F800D911DA39F900DB29F900D9C
:10AB300011240895991B79E004C0991F961708F015
:10AB4000961B881F7A95C9F78095089597FB072E65
:10AB500016F4009407D077FD09D00E94B15007FC8D
:10AB600005D03EF4909581959F4F0895709561951D
:10AB70007F4F0895EE0FFF1F0590F491E02D09948B
:10AB80000E944A51332312F48A1B9B0B0C94CA5522
:10AB90000E944A51B7FF0895821B930B089597FDB9
:10ABA0001094002E083098F00850232F342F452F92
:10ABB000562F672F782F892F912DF4CF15949795C5
:10ABC00087957795679557954795379527950A9572
:10ABD000AAF71124002D08950024A7FD00942A1738
:10ABE0003005400550056005700580059005089505
:10ABF0000F931F93CF93DF938230910510F482E07F
:10AC000090E0E091122EF091132E30E020E0B0E0C1
:10AC1000A0E0309799F42115310509F44AC0281BAA
:10AC2000390B24303105D8F58A819B816115710576
:10AC300089F1FB0182839383FE0111C04081518120
:10AC40000281138148175907E0F04817590799F412
:10AC5000109761F012960C93129713961C933296EC
:10AC6000CF01DF91CF911F910F9108950093122E84
:10AC70001093132EF4CF2115310551F042175307CD
:10AC800038F0A901DB019A01BD01DF01F801C1CF54
:10AC9000EF01F9CF8093122E9093132ECDCFFE01AA
:10ACA000E20FF31F81939193225031092883398356
:10ACB000D7CF2091102E3091112E232B41F42091CB
:10ACC0007128309172282093102E3093112E2091EC
:10ACD0006F28309170282115310541F42DB73EB70A
:10ACE0004091732850917428241B350BE091102E4D
:10ACF000F091112EE217F307A0F42E1B3F0B28173B
:10AD0000390778F0AC014E5F5F4F2417350748F0E4
:10AD10004E0F5F1F4093102E5093112E81939193ED
:10AD20009FCFF0E0E0E09CCFCF93DF930097E9F076
:10AD3000FC01329712821382A091122EB091132E31
:10AD4000ED0130E020E01097A1F420813181820FE5
:10AD5000931F2091102E3091112E2817390709F0DA
:10AD600061C0E093102EF093112EDF91CF910895E2
:10AD7000EA01CE17DF07E8F54A815B819E014115A4
:10AD80005105B1F7E901EA83FB8349915991C40F59
:10AD9000D51FEC17FD0761F4808191810296840F25
:10ADA000951FE90188839983828193818A839B839C
:10ADB000F0E0E0E012968D919C9113970097B9F521
:10ADC0002D913C911197CD010296820F931F2091F6
:10ADD000102E3091112E2817390739F6309751F57A
:10ADE0001092122E1092132EA093102EB093112EAB
:10ADF000BCCFC283D38340815181840F951FC81774
:10AE0000D90761F44E5F5F4F88819981480F591FC0
:10AE1000408351838A819B818283938321153105ED
:10AE200009F0B0CFE093122EF093132E9ECFFD01C8
:10AE3000DC01C0CF12821382D7CF81E090E0F8947A
:08AE40000C942257F894FFCF97
:10AE480001000100010001000100010001000100F2
:10AE580015F118F11CF121F125F19DF134F137F1CB
:10AE68003AF13DF140F129F12BF187F02DF130F164
:10AE780033F136F139F13CF13FF100000000800177
:10AE880000000003000080030000000400001E0012
:10AE980000007A00000072010000E8030000881337
:10AEA80000000000FFFF0100FFFF02000300FFFF9A
:10AEB8000400FFFF05000600070018000C0006004C
:10AEC8000100FFFF0200FFFF03000400FFFF050071
:10AED800FFFF06000700080000000000B609B209DD
:10AEE80000093D90D00380841E90D00324F4000014
:10AEF80024F440420F00127A40420F90D003000021
:10AF080000000000803F0000A040030201000C0D7B
:10AF18000405000000030001020000010100000018
:10AF280000000000000000000000000054F15BF188
:10AF380063F16AF173F17BF182F18AF194F19FF187
:10AF480005040005060204010300010001020302D2
:10AF580001000203040502030504000000001C05AB
:10AF68009C0881046D05B2049004A4042D1A64069B
:10AF7800BE04270900000000C4092D28140AE509A9
:10AF8800C509180BC70ABC291E0A680B620B7B2867
:10AF98005A0B00000000E60CC10C2A1A970CBA0CD8
:10AFA800A70C980CB70D720D650D610D280D090DD4
:10AFB800010D370D2F0D700C6B0C20100120400473
:10AFC800100208010201020408040201040810200A
:10AFD8000408201002020005020105000401010412
:10AFE8000404030303030505030300000101000033
:10AFF8000000D3169C082A1A291AEC1090144D1434
:10B00800E4136313A4137F197F146B10CF108112FC
:10B01800F21270127C180418A517D128610F2B00A2
:10B02800202000202030006F6666005365742000E1
:10B03800536574207377696E6720002D002A004DD0
:10B04800756C74697374657073004D6963726F749D
:10B05800696D696E6773005B005D005365742073EA
:10B06800746570733A005374657020312073657489
:10B07800004446414D205468696E670076312E3988
:10B0880000436F6E66696775726174696F6E00530D
:10B09800637265656E73617665723A00436F6C6FB3
:10B0A80075723A00416C6C6F7720666173743A0070
:10B0B800496E76657274204C43443A005050514EA4
:10B0C8003A004D4944492063683A0043616C69621B
:10B0D8007261746500506C6179204332004F4B20D7
:10B0E80028002900506C6179204334004F4B0044FC
:10B0F8006F6E65004661696C656400536574207302
:10B10800746570733A200042504D3A20004F6E002B
:10B118004F666600426C75650052656400416C6C50
:10B12800003700380031300031310031320031331E
:10B1380000313400313500313600496E742E004537
:10B1480078742E004D494449003234004E6F726DB8
:10B15800616C005265766572736500426F756E6347
:10B1680065004F64642F4576656E005368756666A2
:10B178006C650052616E646F6D004356204D6F64BC
:10B1880065004D494449204D6F646500536574203E
:0DB19800737465702031005377696E670095
:10B1A5001027FFFFFFFF3C028B011851F133F140DF
:10B1B500F10024F400015A00010200FFFF000080A5
:10B1C5003F01000100010001000100010001000133
:10B1D500000000803FFFFF01000048430000080019
:10B1E50000000100000000780000000000000100E0
:10B1F500020003000400050006000700000000002F
:10B20500000000FFFFFFFF0100000001000000003B
:06B2150000142E80000071
:00000001FF
